:020000040000fa
:080000000002040000000000f2
:020000040000fa
:100400000f112200007f2200000188000000000080
:100410000c000700a0d824000100200011000700f4
:10042000000020000000e000020032000000020096
:100430000000000002510200000000000040da004d
:100440000000fe004440a900204f20000000e00012
:100450000300320000002000a00188004440a800f2
:100460000000060091018800800078000000eb0089
:1004700015003700e280400032a0b4009101ba00bc
:10048000e280400032a0b4009102ba00e280400055
:1004900032a0b4000002eb00472bde00f507b200eb
:1004a000602ce10004003a000059eb008301e900f0
:1004b000fdff3e00040037006128e100010032002a
:1004c0000082eb00040007001101ba000200e00006
:1004d000e8ff3a00000006003159ba008301e90044
:1004e0000c0032002159ba008301e90008003200f3
:1004f0000400e00003003a00e280400032a0b400b3
:10050000f5ff370011d9ba008301e900faff3a007c
:100510008100e800e180400032a0b4000000060045
:1005200000000000000000000000000000000000cb
:1005300000000000000000000000000000000000bb
:1005400000000000000000000000000000000000ab
:10055000000000000000000000000000000000009b
:10056000000000000000000000000000000000008b
:10057000000000000000000000000000000000007b
:10058000000000000000000000000000000000006b
:10059000000000000000000000000000000000005b
:1005a000000000000000000000000000000000004b
:1005b000000000000000000000000000000000003b
:1005c0000000000000000000ec874700889fbe008c
:1005d0008a9fbe008c9fbe008e1f7800f0b79f00e0
:1005e00081bf9f008204780000047800010037007a
:1005f0000804e800184778000e00fb00d60007004a
:100600000000e000faff3a00d0c2b300804f57006c
:100610000500320000c0e900804f570002003200a0
:1006200000477800010037000804e8000900e000f6
:1006300045003500e18f54004300320040022000a5
:10064000808f540040003c000900e0000e003400a0
:10065000f08f54001a003a0000c3b300984f100006
:1006600016003a009840900080c7b30080cf500039
:100670000300320080c5b30080cf50000f003a0065
:100680000884e8000e003700a900200000c3b30072
:10069000984f10000a003a009840900080c7b300bd
:1006a00080cf5000040032008900200080c5b300d4
:1006b00080cf500002003a000884e80009012000c1
:1006c0000805780000c3b300010037000a05e80000
:1006d0009a4f1000fdff32008a0578006066b8006e
:1006e0000e003700f0fa210000425200c4ef9f00d4
:1006f0006149b9000c00be00b40e07004fea970034
:100700000401fb00cf91de008b05e800ccb79f0011
:10071000ddb79f0000064100818649001b00fb00f9
:10072000950007008000780009017800f0fa2100a8
:1007300098000700000278000000e000e9ff3a009e
:100740008b0f540006003a000fb897000000e0003d
:1007500029003200ffb0970001087800260037001a
:100760008a805500a0f8210060c07c000000fb00da
:1007700000805000160033004240a9000f003c00ea
:100780004fe997000200fb00cf80de00000056001a
:1007900081805e00800f5600818f5e000700390067
:1007a0006149b900fe0f07004fb19700dfb1970014
:1007b000820f5000838f5800050032002002200075
:1007c000400889000086eb008086eb0005003700ba
:1007d000d0c2b300804f570002003a0060061600f6
:1007e000e0861e008fb997000300e000030032008e
:1007f0008b097800010037006066b8000c00be006d
:100800004f0778004f06be004f05be004f04be00e4
:10081000cf00b10000000600881f780002047800b5
:100820006c000700080040004f047800000006003c
:100830000000fa00881f7800000478003fb9970094
:10084000ea81570080007800c0402000680007005f
:10085000800078000000e000020035000040eb005e
:1008600000f47800010078004f0478000080fa005e
:1008700000000600900178000200e00002003a004b
:100880000308e900050037008080eb001304e00056
:10089000020032000308e8009300fb00010078002a
:1008a000000006000200fa00f0bf9f003fb9970069
:1008b000ea8157008f80e900a0432000050107006e
:1008c0000080fa0000000600800078001106b100e8
:1008d000030035009101b10001003c000050a1006f
:1008e000000006000003b1000b0035009000b100cd
:1008f000080034008000b100070035009001b1000d
:10090000040034007000b100030035009001b10014
:1009100001003c0010000500000005008001780087
:1009200000017800010037000201e8001204e00035
:10093000fdff3a00020037000201e8008100e800f4
:1009400011407800004978000004e000faff3a0006
:1009500003007800000006006900e1000400350093
:100960006d00e100030034000002b100010032001c
:100970000000050010000500800078001104b1009f
:10098000030035009101b10001003c000050a000bf
:10099000000006008001eb00040037008301e8003e
:1009a00090cf1000040032000000e800828f510058
:1009b000faff3a000000eb0000000600300881005a
:1009c0000000e00001003200000001008010220061
:1009d000000006008001eb000200370061f07900a2
:1009e0008301e800828f5100fcff3a0000000600fe
:1009f0006200fa00889fbe008a9fbe000004be000d
:100a0000020578008300780060f92f000f00400095
:100a10007801070088979f0099979f000000eb00de
:100a2000a09f9f009a4578000b80fb000000ea0021
:100a3000cf04de0050c2b30080cf55000200320068
:100a400009047800010037000904e9000800e0000b
:100a50000b0034001f909700080178008a0078008e
:100a60008f9197000300010090979f000000e00025
:100a7000930032002f98970000004400a09f9f0031
:100a80000905450050c2b30080cf55000400320074
:100a90000b04e000e3ff3a002f989700890037002d
:100aa0000000eb00809f9f00f0979f00e0979f0061
:100ab000d0979f00c0979f00b0979f00c09f9f0056
:100ac00009003700c00e22000080500000004000e6
:100ad000010e2200e10078004f989700010070009d
:100ae000c09f9f000a05e8001a4478008800fb00b8
:100af000c00e220044010700800078000000e000e2
:100b0000f0ff3a00a0c2b300804f54000e003a003c
:100b1000bf8897000180e900b08f9f001000780027
:100b2000b09f9f000000e00005003d000000ea00cb
:100b3000b09f9f004f9897000020a000c09f9f008b
:100b40000a05e80010003700b19f9f0003fd2f0049
:100b5000f4ff2700080037003f989700840f5000eb
:100b6000040032006a00b9000000410003004000a8
:100b7000b09f9f000a05e8001a01fb000300410036
:100b8000e90f5000f4ff3600e0c2b3009a4f1000a6
:100b9000040032000080eb00909f9f008a047800e0
:100ba0001c0037008a04e800a0c2b300994f10006f
:100bb00007003a00bf8897000180e900b08f9f00ce
:100bc00010007800909f9f008a84e8001100370091
:100bd0000000eb00909f9f0003fd2f00f4ff270013
:100be000080037001f989700840f5000040032005f
:100bf0006a00b9000000410003004000909f9f0080
:100c00008904e8001901fb0003004100e90f5000ce
:100c1000f4ff3600194478008800fb00e00f220042
:100c2000f90007000000e00002003a0000447800ec
:100c3000010037008904e800a87f9f0080c6b30048
:100c4000804f540004003a00994f14000a003a0003
:100c50006640500006003700c0c6b300804f540005
:100c600005003a00994f140003003a006540400027
:100c7000a07f9f008904e8000905e800c8fb2f0059
:100c80000f04440060f92f000f0040008085e80049
:100c90008801780019417800800078000b00780006
:100ca000ac0107000000e00005003a008800780071
:100cb0000b007800dd0007000000e00059ff3d0058
:100cc0000080eb004f05be004f04be000080fa001c
:100cd000000006001200fa00889fbe008a9fbe0036
:100ce0008c1f780002047800a0b79f00b1b79f0066
:100cf0008300780078805700be0007000000eb00fa
:100d0000e0b79f00d8b79f0000067800dfb49700d7
:100d1000194578000a80fb000000ea00cf05de00dc
:100d20000a00fb000cff07000000e0001a00320080
:100d30006fb097000000e800e0b79f003fb0970059
:100d4000120020008000eb00afb19700030001000b
:100d50000004780000ff0700000178000000e000b8
:100d6000f3ff3a006fb09700e10f44000700320034
:100d70000000e900e0b79f003fb0970088007800ce
:100d8000afb1970003000100230037000000e90025
:100d9000e0b79f002000370050c2b300804f5500dd
:100da000020032000b047800190037000b04e90040
:100db000170037006fb097000000e800e0b79f0011
:100dc0003fb09700120020008000eb00afb1970009
:100dd00003000100800078001900fb00808f5000a4
:100de0000a003200e18f40007c0032006fb09700b3
:100df0000000e900e0b79f003fb097000001eb0062
:100e0000afb1970003000100740037008904e800c7
:100e10000804e900e7ff3b005fb0970080804500d1
:100e2000d1b79f0050c2b300804f5500030032007d
:100e30000a04e000b5ff3a0068003700a2c2b30020
:100e40000040eb00914f110003003a000100e80060
:100e5000d0b79f0002407800a0f79f000000eb0091
:100e600080bf9f0003fd2f00f4ff27000a0037001a
:100e70000fb89700840f5000040032006a00b900d8
:100e8000000041000300400080bf9f005fb097005a
:100e90000000e800d0b79f00dfb497001944780045
:100ea0000801fb0003004100e90f5000f0ff36008d
:100eb00082007800200f2200530007000000e000ad
:100ec00002003a0000447800020037000900e80000
:100ed000d0b79f00b8f79f0080c6b300804f540082
:100ee00005003a00dfb09700914f14000c003a0063
:100ef0006640500007003700c0c6b300804f540062
:100f000007003a00dfb09700914f140004003a0048
:100f100065404000b0f79f000100e800d0b79f0097
:100f20005fb097009000fb00900f22003600070092
:100f30000000e00019003a006fb097000000e800e0
:100f4000e0b79f003fb09700120020008000eb0048
:100f5000afb1970003000100000478007efe070097
:100f6000000178000000e000f3ff3a006fb0970046
:100f7000e10f4400070032000000e900e0b79f00e5
:100f80003fb0970088007800afb1970003000100e0
:100f9000020037000000e900e0b79f007c805700a6
:100fa000690207000000e00003003c000c00e000c4
:100fb00009003200090037004ff097000004e000fc
:100fc000010032000c06e8005fb097000000e80066
:100fd000d0b79f004dff3700000678000c00780066
:100fe0004f0678004f05be004f04be000080fa0097
:100ff000000006000200fa00f1bf9f00010878001f
:101000000080fa0000000600040037000204e0003f
:1010100001003a00000005000000e80010417800df
:10102000814f5100f9ff3a00000006000400fa0069
:10103000889fbe008a9fbe008c1f78000004780045
:101040000106780070089000f80090000100500040
:10105000880890000100500098089000010050009e
:10106000a808900001005000b8089000010050004e
:10107000c8089000810550000002220090bf9f0028
:1010800000032300a0bf9f00081090000028a300c9
:1010900018003a000b00e000160034008b047800c2
:1010a00009057800e28f5400020036002a00200073
:1010b000020037000900e0000b00340058009000e7
:1010c000c80190000a017800ee805700030001007b
:1010d000500498000000e00096003200680890007c
:1010e00000004500600c98008a8454004240a9002a
:1010f000ebff3c00780190000200e0000b003400a0
:1011000058009000c80190008c0078000300010096
:10111000500498000000e00086003200680890004b
:10112000f800900001004000600c9800880c9000ce
:101130000900e0001500340009057800e28f540032
:10114000020036002a002000020037000900e000fb
:101150000b00340058009000c80190000a0178008c
:10116000ec80570003000100500498000000e000ec
:10117000700032006808900000004500600c980084
:101180008a8454004240a900ebff3c0018099000fb
:101190000200e0000b003400e800900058009000ce
:1011a000c801900003000100500498000000e00016
:1011b000600032006808900098089000010040002c
:1011c000600c9800a80c90000900e00015003400a5
:1011d00009057800e28f5400020036002a00200042
:1011e000020037000900e0000b00340058009000b6
:1011f000c80190000a017800ec805700030001004c
:10120000500498000000e0004a0032006808900096
:1012100000004500600c98008a8454004240a900f8
:10122000ebff3c00380990000200e0000d003400a4
:10123000e80090001808900080804000580090005e
:10124000c801900003000100500498000000e00075
:101250003800320068089000b80890000100400093
:10126000600c9800c80c90000900e00015003400e4
:1012700009057800e28f5400020036002a002000a1
:10128000020037000900e0000b0034005800900015
:10129000c80190000a017800ec80570003000100ab
:1012a000500498000000e00022003200680890001e
:1012b00000004500600c98008a8454004240a90058
:1012c000ebff3c00081090000028a3001b00320038
:1012d0000b00e000190034008b0478000905780049
:1012e000e28f5400020036002a002000020037007e
:1012f0000900e0000b00340058009000c801900085
:101300000a017800ee8057000300010050049800a5
:101310000000e0000700320068089000000045006f
:10132000600c98008a8454004240a90003003400f5
:10133000eaff37000080eb00010037000000eb00ff
:101340004f0678004f05be004f04be000080fa0033
:1013500000000600889fbe008a1f78000004780005
:1013600001027800824478000305780070c6b3005b
:10137000804f510021003c0000c0e900804f510027
:10138000de003d0072405000804f51004b013200a2
:101390000d003c006c405000804f51005e013c004d
:1013a00000c0e900804f5100d4003d0050c2b3009e
:1013b000804f5100550132007c404000804f510069
:1013c00055013a00cd00370010c6b300804f5100e0
:1013d000ca00320004003c0069405000804f5100b8
:1013e0004d013a007200370030c6b300804f510003
:1013f000180032000040e8000900370000c7b300c1
:10140000804f51001e01320008003c0000c0e9007e
:10141000804f5100e400320065003c006540500000
:1014200080cf54003c013a000f00370050c7b30092
:10143000804f51005e00320063404000804f5100f9
:101440005b00320065405000804f510032013a008d
:101450001a0137009180e900010a780078009000b5
:101460009171780032013700a8609000c0c6b300c7
:1014700080cf50000a003a00940078006480500049
:10148000000a78001000be004f89de00cf91de0018
:101490000002be00020378008203780013003700c8
:1014a00010c7b30080cf500003003200a0c6b300c5
:1014b00080cf500006003a00940078006880500009
:1014c000000a78003002be002003be00070037008b
:1014d0001480e900000a780010007800000278000b
:1014e000cfa2de000503780086037800049cbe00ce
:1014f0000694be00a860900080c6b30080cf500064
:101500000e00320020c6b30080cf500005003a0024
:101510000400fb00cf80de0001017800820178002a
:101520000a00370040c7b30080cf500003003200ec
:101530006640400080cf500006003a00040078006a
:10154000cf80de000101780082017800009cbe009f
:101550000294be003800be002801be00e00f50001b
:10156000e08f5800e00f5900e08f590003003d0064
:1015700078009000d1c2b3000a0037000810900034
:101580000018a3000300320078009000b1c2b3003d
:10159000040037000008a3005300320078009000d8
:1015a00001c2b300017578000000e8004d0037006b
:1015b000a8609000c0c6b30080cf500006003a007b
:1015c0009400780064805000000a78001002be0089
:1015d0006033b8001300370010c7b30080cf50004d
:1015e00003003200a0c6b30080cf500006003a00ce
:1015f0009400780068805000000a78003002be0035
:101600002003be00070037001480e900000a7800bc
:10161000100078000002780005002000060020007d
:1016200007002000049cbe000694be00a860900045
:1016300080c6b30080cf50000e00320020c6b30039
:1016400080cf500005003a000480fb00010020001c
:1016500002002000030020000a00370040c7b3004a
:1016600080cf5000030032006640400080cf500021
:1016700006003a000400780001002000020020006b
:1016800003002000009cbe000294be0008109000e1
:101690000038a300140032003800be002801be004c
:1016a000e00f5000e08f5800e00f5900e08f590024
:1016b0000d00320080c7b30080cf54000300320019
:1016c00080c5b30080cf540007003a007800900036
:1016d00001c3b300017578008000e80009f57800c7
:1016e0000080e80070049800780090000000450039
:1016f00060049800894078006d003700a860900071
:10170000c0c4b30080cf500006003a0094007800b7
:1017100068805000000a78005001be004000be0002
:10172000050037009400780064805000000a7800bb
:101730001000be002a0c0700009cbe000294be00f0
:10174000380090000000e00003003d0078009000a9
:10175000d1c2b3000a003700081090000018a3009f
:101760000300320078009000b1c2b30004003700db
:101770000008a300050032007800900001c2b30009
:10178000017578000000e80070049800780090006f
:101790000000450060049800894078000800780047
:1017a0009002070064003700a8609000c0c6b30034
:1017b00080cf5000250032000a003c0064405000f9
:1017c00080cf50002800320000c0e80080cf5000d9
:1017d000140032006840500080cf500022003a00d0
:1017e0000a00370040c7b30080cf50001e0032000f
:1017f0006640400080cf50001b003200694050001e
:1018000080cf500018003a00060037001480e9002d
:10181000000a780010007800485c900008487800c2
:10182000450037001480e900000a780010027800b3
:1018300068089000cf80de00010178008201780006
:10184000009abe000292be003b0037001480e900ff
:10185000000a78001001780068089000cf80de0050
:101860000089be00340037001480e900000a7800c7
:1018700010007800680c9000080878002e003700ef
:101880001180e9008008780010007800cf80de0029
:101890000101780082017800009cbe000294be0025
:1018a00078009000000045006004980081c7b300f4
:1018b00008007800bb0007001f0037001480e90013
:1018c000000a780010007800600498005809900021
:1018d0000200e00002003d003b0207000900370063
:1018e0008000eb002bfc0700800078000000e00087
:1018f00003003200680090000080500001003700b3
:1019000058089000100c98000b00370078009000e9
:1019100002757800060037007800900080004500ce
:101920000904e00001003a0059c2b3008948780078
:101930000000e800700498000000eb004f057800fc
:101940004f04be0000000600881f780000047800e5
:101950000040eb0000549800380090009040780060
:1019600090c6b30080cf50002a00320013003c0024
:101970007140500080cf50002600320005003c002e
:1019800050c2b30080cf50006400320030c5b300b5
:101990001b00370030c6b30080cf50001b00320060
:1019a0000040e80080cf50001a003200694050002b
:1019b00080cf50006e003a007300370000c7b300bc
:1019c00080cf500007003c000040e90080cf50006d
:1019d00010003d000040e90080cf500064003a0054
:1019e0000f00370050c7b30080cf5000090032000d
:1019f0006340400080cf5000060032006540500038
:101a000080cf500043003200590037008000eb00c7
:101a10005e003700080078001b0407005f003700f5
:101a2000684890000004e0005b003a00f84890002d
:101a3000c0c6b30080cf5000270032000a003c002f
:101a40006440500080cf50002b00320000c0e800fe
:101a500080cf5000150032006840500080cf500009
:101a600025003a000a00370040c7b30080cf50007d
:101a7000210032006640400080cf50001e0032003e
:101a80006940500080cf50001b003a00070037002b
:101a9000280090000080e9002004980010007800e1
:101aa000084c9000084878003b0037002800900060
:101ab0000080e9002004980010027800480090009f
:101ac000cf80de000101780082017800009abe001c
:101ad0000292be0030003700280090000080e9002c
:101ae000200498001001780048009000cf80de00ac
:101af0000089be0028003700280090000080e9001f
:101b0000200498001000780048049000080878002d
:101b100021003700110020001c0037004800900011
:101b20000000e80040049800180090009801780038
:101b3000120020008000eb0003000100800078000c
:101b400050022000808f50001300320048009000a7
:101b5000e18f4000080032000000e90040049800d6
:101b600018009000980178000001eb0003000100cc
:101b70000000eb00090037000000e9004004980075
:101b800001007800050037008080eb000800780035
:101b90001605070001003700100020004f047800f0
:101ba000000006002f03b000889fbe008a9fbe0081
:101bb0008c9fbe008e1f780000077800f00c22007a
:101bc000c0b79f0080c5b30080cf5000080032002e
:101bd000e20b2200c2b79f007740400080cf500048
:101be00003003a0083002000b3b79f000a003700cb
:101bf00080c7b30080cf500005003200a400200051
:101c0000b4b79f0080c5b30080cf500002003a00f7
:101c100005012000b5b79f003e04be002e05be00a2
:101c200040c6b30080cf5000030032006540400042
:101c300080cf50000b003a00e00f5400e08f5c00b2
:101c4000e00f5d00e08f5d0006003d006000b80021
:101c50006011b80008045000898458000a05590032
:101c60008b855900bfb39700e88f53000300320003
:101c7000f08f530045003a00020037003600200084
:101c80000100370046002000e00f5400e08f5c00a8
:101c9000e00f5d00e08f5d0005003a005e089000f7
:101ca00081012000a1b79f000000e0000800320081
:101cb0003fb197000200e90008006000cfb1970033
:101cc0006340780090df9f0074012000a4b79f005c
:101cd000860278008502e900050033008b05d100fb
:101ce0000a85d3008984d3000884d300f9ff370024
:101cf000089fbe000a97be00afb397000700e90037
:101d000021fc2f008f804000008240003fb19700ef
:101d10008202e90012003700afb397008703e900a1
:101d2000a7b79f0000806200cfb097006152780093
:101d30003e00be002e01be00860378008703e90046
:101d4000050033008381d1000281d3008180d3005c
:101d50000080d300f9ff3700009fbe000297be004d
:101d60003e00be002e01be00e00f5000e08f580084
:101d7000e00f5900e08f5900d6003400afb3970050
:101d80000700e000e4ff3c00d2003700ae609000a6
:101d900080c6b30080cf50000b00320006003c002c
:101da0000104e000080032006640500080cf50007f
:101db00073003a0004003700c0c6b30080cf500063
:101dc0006f003a0031003700080178000800e00099
:101dd00005003a005e08900081012000a1b79f0035
:101de0000000e00009003200bfb1970011000900b7
:101df0000381d8008000fd004fb297006440780056
:101e000090df9f0075012000a5b79f00bfb397002a
:101e1000110009000781d80080017800afb0970059
:101e20000100e90022fc2f000f01410000024100e7
:101e30000c003700bfb29700110009008501d800df
:101e400000017800afb397008703e900a7b79f00b0
:101e50000590b90000805100cfb097006152780022
:101e6000820178000300e000030034002fb19700e6
:101e70000200e000efff3c0003007800cf80de00ae
:101e800001017800820178003a0037000806be00a0
:101e9000e00f5400e08f5c0005003a005e089000ff
:101ea00083012000a3b79f000000e000090032007a
:101eb0003fb297006121b9000c00be00670a07001d
:101ec000cfb297006540780090df9f007701200037
:101ed000a7b79f003fb297006121b9000c00be0078
:101ee0002f0a07000006be00afb297000500e90008
:101ef00027fc2f008f8343008083430097b79f0008
:101f0000110037003fb197006114b9000801be000d
:101f10000c00be00540a07000005be00afb19700d8
:101f20008301e900a3b79f000801be00a7080700ce
:101f3000000056001fb29700cfb29700655278009c
:101f400094b79f000a06be00e00f5600e08f5e00c7
:101f500003003400afb397000700e000e9ff3c0046
:101f60004feade00cfa2de000c00be0004017800c4
:101f700084017800009fbe000297be005500370024
:101f8000e00f5400e08f5c00e00f5d00e08f5d002b
:101f900005003a005e08900081012000a1b79f0073
:101fa0000000e0000d0032003fb19700020278000f
:101fb000cfa2de0005037800860378000800be008b
:101fc0000a01be00b80a07004fb2970064407800cb
:101fd00090df9f0075012000a5b79f003fb19700db
:101fe00002027800cfa2de000503780086037800a5
:101ff0000800be000a01be00a40a0700009fbe0040
:102000000297be00afb197000300e90024fc2f0047
:102010000f0242000006420020003700bfb29700c6
:1020200005047800cfc4de00090578008a05780031
:102030000802be000a03be005fa89700efa8970041
:102040007fa997008fb197009b0a0700d0b79f0028
:10205000e1b79f00f2b79f0083bf9f00afb3970027
:102060008703e900a7b79f000802be000a03be006d
:10207000170b07005faa970000005200cfb297002d
:10208000655678005fb09700efb097007fb197007a
:102090008fb99700009fbe000297be003e00be00b1
:1020a0002e01be00d0af9f00e1af9f00f2af9f00b6
:1020b00083b79f00e00f5000e08f5800e00f5900f9
:1020c000e08f590003003400afb097000100e0003a
:1020d000d2ff3c003fb19700e80f510013003a00d7
:1020e0000e1090000038a30010003200afb197002e
:1020f000f78f510006003e0024fc2f000f02420023
:102100008300420000c3b300914f1000070032006b
:10211000afb297008502e900a5b79f0000c3b300e6
:1021200027fc2f008f83430080f37a00afb1970024
:1021300078811100120f98006e00900024fc2f008f
:102140000f0242008300420022fa07001e0990009d
:102150005e089000800f510006003d000200500014
:10216000000f98000e1090000040a100001798008a
:102170000f0037000000e0000d003d000e10900041
:1021800074006000f00f500009003a007e089000d3
:10219000fe009000010050008e08900001005000e9
:1021a000020050004240a90001003400000f9800d6
:1021b0004f0778004f06be004f05be004f04be001b
:1021c0002f03b100000006008000780001003700f6
:1021d0000000e8001004e000fdff3a00010050009c
:1021e000000006008f04b000889fbe008a9fbe00da
:1021f0008c9fbe008e1f7800f0b79f0081f79f0074
:102200005001be004000be00f0979f00819f9f00dc
:10221000929f9f00a39f9f0010c6b3000ff19700ed
:10222000804f51001600320010c4b300804f51009f
:1022300013003200ffb19700530890000000e00047
:1022400003003d0060002000d00998000c0037001a
:102250000000e0000a003a0070c6b3000ff29700d9
:10226000804f52000300320070c4b300804f520010
:1022700003003a0010002000ffb29700d00a980037
:10228000ffb09700c0fa2f000f0040004404070081
:1022900080017800e20f500015003a003000200065
:1022a000ffb097009008980010c6b3000ff1970098
:1022b000804f51000a00320064404000804f5100be
:1022c000070032000040e800804f51000400320057
:1022d000610622000040e800804f510001003a00f2
:1022e000a1062200ffb1970063009000160037009e
:1022f0000000e00018003400300020007fb297009a
:10230000100a980010c6b3008ff2970080cf5200d9
:102310000a0032006440400080cf520007003200c3
:102320000040e80080cf520004003200e1062200a5
:102330000040e80080cf520001003a00210722004f
:102340007fb19700620090003158780031587800d2
:1023500011487800c601370014c6b3008ff2970009
:1023600084cf52000300320010c4b30080cf52006b
:1023700013003a007fb0970060019000820078005f
:1023800000c3b30080587800ffb29700e1029800c4
:1023900080c7b3008ff2970084cf52000100320053
:1023a00080c5b300804878000280e800ffb0970045
:1023b000e0009800710090000080e800f0009800b4
:1023c0000300e00005003a00e3979f0064fb2f0044
:1023d0000f01420003077800a001370065072200c3
:1023e000e5b79f0010c6b3008ff0970080cf500074
:1023f0000500320010c4b30080cf5000a7003a009f
:1024000072082200e2b79f00ffb1970053089000c6
:102410001e0220000000e000010035000007e80077
:102420000e02e800d4b79f006022b8006033b80005
:102430007f9097008f9897001f999700af9997000a
:10244000510a0700ffb097003102be002103be0011
:102450000000e00004003d000400be000601be00d4
:1024600003f0a200020037000400be000601be0017
:10247000f0979f00819f9f00929f9f00a39f9f00c6
:102480006f91970064015100e2979f00c3fa2f00fb
:102490008f8141006a8041000048eb006b8241005f
:1024a000c4b79f0031003700c201200003002000a4
:1024b000e5fa2f000f804200e50307007f949700a4
:1024c0008f9c97001f9d9700af9d97000800be004e
:1024d0000a01be00310a07000006be005fb1970086
:1024e00067015100d2b79f004240a9000a003400a2
:1024f000560a07000002be000203be000800be002c
:102500000a01be00540a0700f0979f00819f9f00b8
:10251000929f9f00a39f9f00cfb1970067804100cb
:1025200071002000050037006f6066004c6add0016
:102530004466de000c067200c4eede00e00f5600ba
:10254000e08f5e00050034008100e900e18f40006b
:10255000f5ff3a00010037000060eb008100e90060
:10256000fdff3b0067004000c0b79f00dfb297004f
:102570000500e000090034006022b8006033b800b4
:102580007f9097008f9897001f999700af999700b9
:10259000330a07000000e000c3ff3c0060fb2f008f
:1025a0008f0040004fb19700010051000000e9008a
:1025b0008e0f500001003d00000778000e00e00083
:1025c00003003d0073fb2f000f8141002c003700fa
:1025d000800f570005003d000e8040001040900025
:1025e000f3c0b300e74f500001003c008041eb0016
:1025f000c4fa2f000f0242000e0042006a004000a1
:102600008e007800010037000000e9008100e90039
:1026100010417800834f5100fbff32000107e800b2
:10262000efcf510001003a000248e8000100e0004d
:102630000300350075fb2f000f81420006003700b4
:102640000e07e8006f90970064004000e0979f003d
:1026500061fb2f000f8140008e0041008e01780049
:10266000030037001100fb006fb29700e4487800c8
:102670008301e9008100e9000300e000f9ff3d006b
:10268000ffb29700550890000000e000f3003d0005
:102690000e00e900d00a9800f00037007f94970000
:1026a0008f9c97001f9d9700af9d97006022b800f8
:1026b0006033b8000800be000a01be00b20907007e
:1026c0000000e00005003d000bf0a200f8979f001d
:1026d000899f9f009a9f9f00ab9f9f006f909700dc
:1026e000725927000280b900026a280013002000f6
:1026f0005d080700e4005000e1979f0015003b00d3
:10270000e3801000c0ff2f00008460000800ea0092
:10271000e0979f007f9097008f9897001f999700f0
:10272000af999700e9012200070037000808a300cd
:10273000030032003902be002903be00cd090700a4
:102740000884d100e88444000800e000f7ff3c0062
:102750001b0037000100e0001d003400c0ff2f0007
:1027600000806000e0979f00000478006000b800df
:102770000200200003ff2300e901220007003700c8
:102780000808a300030032003902be002903be007e
:10279000b80907000884d100e88444000800e0007c
:1027a000f7ff3c000002be000203be007f909700ce
:1027b0008f9897001f999700af999700220a0700fa
:1027c000f0979f00819f9f00929f9f00a39f9f0073
:1027d000ffb097005109900060c6b3008ff19700d9
:1027e00080cf5100040032006100200060c4b300bb
:1027f00080cf510002003a006f929700ea00420039
:1028000001074100f30f5700010034003e01200092
:1028100000c3b300e0779f0075fb2f008f8242005a
:10282000b5b79f00330037000800be000a01be00a4
:102830005a0907000006be00680757004240a90079
:102840000e003400810907000002be000203be0032
:102850000800be000a01be007f0907006022b80020
:1028600046782d007719240082090700f0979f0011
:10287000819f9f00929f9f00a39f9f003fb0970062
:1028800068044000890020000d003700a4002000eb
:10289000050020000c01be00e0fd2f000f004000ed
:1028a000660307007fa897008fb097001fb19700bd
:1028b000afb1970004c3b300046441000006be003a
:1028c000e00f5600e08f5e00060034008904e90046
:1028d000e18f4400edff3a000200370000c3b3006f
:1028e000006478008904e900fcff3b0068044400b0
:1028f000b8b79f000e00e0000b0034007f949700f3
:102900008f9c97001f9d9700af9d97006022b80095
:102910006033b8000800be000a01be00500907007d
:102920000000e000c0ff3c00c5fa2f008f8242008b
:102930006a804200bfb09700008050008001e9002b
:102940006f919700e70041006b81420000c3b30024
:10295000010037000201e800924f1000fdff320035
:1029600074fb2f000f0042008080400082805000e6
:102970000080410002025000e1979f00ffb29700e3
:10298000d509900060c6b3008ff2970080cf520047
:102990000300320060c4b30080cf520002003a004e
:1029a0008100e8000a00370050c6b3008ff097009e
:1029b00080cf5000050032008000eb0050c4b3000f
:1029c0008ff2970080cf520001003a0011002000e2
:1029d000018741008e0f520001003d00040778007e
:1029e0000e00e0001d003500840f570005003d007b
:1029f000e2407f0095c3b30040c3b30080cf5000d6
:102a000001003c0005c3b3000e0041008000e90056
:102a10008e017800010037008100e9008301e900a0
:102a200011427800854f5200fbff32000307e80097
:102a300090c3b30080cf520001003a008448e80000
:102a40000300e00005003d000201e9000e07e80078
:102a50006f9097000000e800e0979f006f9297004a
:102a60008e0178008ff097007fb097001003070069
:102a70004f0778004f06be004f05be004f04be0052
:102a80008f04b100000006002f02b000889fbe0036
:102a90008a9fbe008c9fbe008e1f78008004780045
:102aa000600090000000e00001003c00f0ff270003
:102ab0000000e900d0049800c90090000c00330029
:102ac0000100e800c0049800190090009901780006
:102ad000120020008000eb000300010000057800d8
:102ae000b0022000800f550006003a000b003700ae
:102af0000100e800c00498002cfd2f000f064600de
:102b00001b003700d0022000800f55000300320068
:102b10002cfd2f000f0646001600370030fd2f0059
:102b20000f044000aad79f00590090000000e90060
:102b3000d0049800c90090000a0033000100e800aa
:102b4000c00498001900900099017800120020003c
:102b50008000eb0003000100000578000806780003
:102b6000040037000100e800c0049800080678005f
:102b70000085eb00f8092200390090009000fb006e
:102b80000800780020f907000800500081092200a1
:102b9000614478008805fb0000032000800f550089
:102ba00033003a00590090000000e900d00498007a
:102bb000c90090000c0033000100e800c004980038
:102bc0001900900099017800120020008000eb00ad
:102bd000030001000005780080072000800f5500e9
:102be00005003a00070037000100e800c004980023
:102bf0000085eb001b00370080052000800f55008a
:102c000018003a000804e00002003200f04f5400bf
:102c10001d003a00590090000000e900d00498001f
:102c2000c9009000090033000100e800c0049800ca
:102c30001900900099017800120020008000eb003c
:102c40000300010000057800030037000100e800e0
:102c5000c00498000085eb000047eb000b0120004a
:102c6000110037000804e000b80032000600370009
:102c70000047eb000804e00004003a00ad0020002b
:102c8000084778001c0037001ec0b300ad002000cc
:102c9000ea4f540018003200e88f550002003a0055
:102ca0008b067800140037006d01200012003700f9
:102cb000590090000000e900d0049800c90090007d
:102cc000090033000100e800c004980019009000da
:102cd00099017800120020008000eb000300010041
:102ce00000057800030037000100e800c0049800e8
:102cf0000085eb001ec0b30000032000800f5500cc
:102d0000ebff32000e04e00018003200005e780095
:102d1000160037006f805700800f56000100310009
:102d20000a5e7800590090000000e900d004980085
:102d3000c9009000090033000100e800c0049800b9
:102d40001900900099017800120020008000eb002b
:102d50000300010000057800030037000100e800cf
:102d6000c00498000085eb001ec0b300e10f4500d1
:102d7000070032000d0178008a007800700a2200f6
:102d800004f707000000e000e2ff3a0066003700a9
:102d9000490090000000e900c00498000e04e00023
:102da00008003a0020fd2f000f004000800f560061
:102db0005b003a00e10f450059003a008a007800b4
:102dc00065003700004eeb006948900011002000bc
:102dd0000004e00060003a00390090009040780064
:102de00040c6b30080cf5000030032006540400071
:102df00080cf50000a003a000b0178008000eb0001
:102e000020fd2f000f0040005d0307000203be00fd
:102e10000002be0010c0b300805498000d003700bf
:102e20000b0178008000eb0020fd2f000f00400018
:102e3000ad0307000203be000002be0010c0b300d5
:102e400080549800b900900000c7b300914f100063
:102e50002c003200f9489000c0c6b30080cf50006b
:102e6000220032000a003c006440500080cf500035
:102e70002400320000c0e80080cf5000140032006f
:102e80006840500080cf50001e003a000a00370012
:102e900040c7b30080cf50001a00320066404000a7
:102ea00080cf5000170032006940500080cf5000a2
:102eb00014003a0006003700290090000080e90065
:102ec000a004980010007800044878001200370031
:102ed000290090000080e900a0049800100078000c
:102ee0000498be000690be000b0037002900900039
:102ef0000080e900a0049800100078000488be005b
:102f000005003700290090000080e900a004980027
:102f10001000780004087800110020000e0037002f
:102f20008000eb000c003700490090000000e90031
:102f3000c004980019009000990178000001eb008e
:102f40008a0078000300010094ff37001ec0b30020
:102f50008b00200052ff3700010078004f077800f7
:102f60004f06be004f05be004f04be002f02b10049
:102f70000000060080017800d4c2b3000f003700c3
:102f80000300e800904f120008003a0093cf1000b1
:102f900003003e002340900080cf50001200360016
:102fa000e3814100630151000400370093cf10001a
:102fb0000d0032000201e90080017800e20f5100ab
:102fc000efff3e000002eb000400370064c0790010
:102fd0000402e800814f500003003200820f5200cb
:102fe000faff3a000000050010000500f0874700d6
:102ff000889fbe008a9fbe008c9fbe008e1f7800f7
:1030000000047800810678000000eb00c0b79f0044
:10301000f8489000c0c6b30080cf500002003a00cc
:1030200011002000c1b79f000d00e00023003d000b
:10303000b80090000100e80030049800e2c5b30039
:103040008041eb0083f79f00904f110003003a008e
:103050000180e8003004980082f79f00b8049000d7
:10306000d0c5b300994f100002003200090078006b
:10307000010037000900e800d1052000e2f7070051
:10308000d0b79f008000eb000000e000bd003200e0
:1030900009065000e20f5600080034000c81e900d8
:1030a0000900e800d10220003af6070011c0b30081
:1030b000c1ef9f000000e00002003a008041eb00f9
:1030c000c3ef9f00680090000000e00004003c0097
:1030d000f0ff27000d00e00001003a001000200082
:1030e00050049800684890000004e0000d003a0089
:1030f00028009000cfb097000100e00005003200ea
:103100000080e9002004980010007800b0b79f000c
:10311000040037000080e9002004980010007800c7
:10312000f0b79f000045eb005e0037000d00e000a7
:10313000030034000900780007f607001e0037007e
:103140000d00e0001e003200cfe997000304e0000c
:103150000c003a00380090008ff097000104e00066
:1031600004003a000c0178008900780009f6070095
:103170000b0037000c0178008900780005f6070085
:103180000d003700380090008ff197000304e00035
:1031900006003a000c0178008900780075ff0700ee
:1031a0000000e00006003a006d0037000c017800d6
:1031b000890078006fff07000000e00068003a0017
:1031c0004fb097000000e00009003a006848900006
:1031d0000004e00032003a00ffb097008958780000
:1031e000f1b79f0010c0b300005498002c003700c6
:1031f000c9e79f008905fb000b0078000100320041
:1032000010002000000578001e0020000000e000f3
:1032100016003a000904e00004003a007c805700e0
:10322000e9fb07000005e800100037000e07e90081
:10323000fc81570063407f008000fb004801900044
:10324000e14f4000070032000200e900400498000e
:1032500018009000980178000001eb0003000100c5
:10326000020037000200e900400498008e0f55006c
:10327000eeff3500684890000004e00005003a00c9
:103280003fb097000b187800b0b79f0010c0b30094
:1032900000549800680090000000e9006004980065
:1032a0002ac0b300580090000000e90050049800c4
:1032b000480190000b0033000200e8004004980031
:1032c0001800900098017800120020008000eb00a8
:1032d0000300010080047800e10f400093ff3a00f2
:1032e000020037000200e800400498004800900007
:1032f0000000e900400498000d00e00002003200e8
:10330000e24f5500040032000a00fb008080eb0011
:103310001c00320010003700684890000004e000f4
:1033200009003a00cfb097000100e000030032002e
:10333000bfb197008009eb00030037008fe89700ca
:103340007fb09700014878000d00e00002003d00ca
:10335000dfb1970033049800110020000900370006
:10336000480090000000e900400498001800900018
:10337000980178000001eb0089007800030001004b
:10338000ddff3700010078004f0778004f06be00d0
:103390004f05be004f04be000f01b1000000060043
:1033a000889fbe00800478006684400000ff2700ec
:1033b000180060004401de00f07f2000800f510003
:1033c0000e003a00800ceb00180478006f006400d7
:1033d0001c003a00210090000000e00019003a00b3
:1033e000110090000000e00016003a0010002000dc
:1033f0001100e00014003200120037000200e0006b
:1034000005003c0001007800190307000001780066
:103410000000e00008003c00f000280018006000f8
:1034200001fe2300010c700020c02f00800c410021
:103430000080eb0004003700800ceb000000eb0084
:1034400001003700200020004f04be0000000600ed
:10345000889fbe008a1f78008c9fbe000004780001
:103460000206be00e6044000190178000200d00008
:103470004505de008a007800f07f2000800f5500af
:103480000c003a006f00610067003a0028009000cd
:103490000000e00064003a00180090000000e00026
:1034a00061003a00100020001800e0005f003200c8
:1034b0005d0037000a00e00007003a0008007800cd
:1034c000eb020700800078000000e00002003400fa
:1034d0000a007800550037006108b9000c0140006f
:1034e0008d814800e07f2000800f5100e08f59005f
:1034f0000d0034001900e00004003d006000b80039
:103500000200200003ff2f00030037006000b80016
:103510000200200003ff2700009cbe000294be00b2
:103520001000200041003700e00f5100e08f5900eb
:1035300005003400f000280019006000c410dd0010
:10354000810c700036003700190078000100280057
:10355000010360006f0060000040a000800c780054
:1035600061015100e0815900c0fc2f00f1ff2f00e4
:10357000800f5100818f590006003d00860c7800b5
:103580000000eb002004980010049800000c780064
:1035900026003700020078000881e800e4004400bb
:1035a00005003700120c780011097800990878009e
:1035b000800ceb0070004000f00f4000f9ff340079
:1035c0008002ea00150032008881e8007082120053
:1035d000980078008508de00130078000400dd0004
:1035e000008c700064014400930078008508de00c0
:1035f000120078000400dd008089700092007800dd
:103600008508de00190078000400dd0000897000e4
:10361000190078000500de00800c7800990c73001a
:103620000080eb0001003700200020004f06be00a4
:103630004f0578004f04be00000006000400fa00a9
:10364000889fbe008a9fbe008c1f7800000678000d
:1036500092bf9f00a3bf9f000404be000401be00f0
:103660001fb89700afb897007f0407000005be00a1
:103670000001be000800be00d40207001fb9970079
:10368000afb99700000051008180590020069800d2
:10369000310698000a8ebe000c0078004f067800b4
:1036a0004f05be004f04be000080fa000000060077
:1036b0000e00fa00889fbe008a9fbe008c9fbe004d
:1036c0000004780001457800020678008304780041
:1036d000840678000300e00002003c00190020008e
:1036e000cc10220060c6b300804f55000e0032009f
:1036f00060c4b300804f55000b00320070c6b300a9
:10370000804f55000300320070c4b300804f550055
:103710009c003a00e48f4600800035005808900075
:10372000808f56007d003d008d05e80060c6b30027
:10373000804f55001000320060c4b300804f550028
:103740000d003200081090000038a30004003a0079
:1037500058089000808f540001003d00590c9800db
:10376000580890000b005000500c980002003b00dd
:103770000000eb00500c98000b00e00027003c001c
:10378000180990006800900001c3b300017079002f
:103790008201e800130c9800580890000000e00037
:1037a00003003c00081090000038a3000500320020
:1037b00068009000e1c2b30001f079000280e800e7
:1037c000100c9800d80890000b00ea00808f500081
:1037d00001003d008105ea000b00ea00200c980082
:1037e00001804500500c9800890f500001003d00f9
:1037f00080047800390c98006800900098089000c8
:1038000001004000090178008c00780071f4070085
:1038100058089000090050001a00370098089000de
:10382000680090008b8f540018003d00010040009c
:10383000090178008c00780066f4070018089000f1
:1038400000814400120c980009805500200c98005b
:10385000580890000000e00003003c0008109000b1
:103860000038a30006003200e8009000e0c2b30078
:1038700080707900380890000000e800300c980053
:1038800058089000400c9800a60037000100400046
:103890000b0178008c0078004ef4070018089000a7
:1038a00000814500120c98008b8454005808900049
:1038b0000000e00003003c00081090000038a30066
:1038c0000500320068009000e1c2b3000170790089
:1038d0000200e800100c980058089000890f500072
:1038e00001003d0080047800680090009808900076
:1038f000010040008b0046000901780035f4070004
:103900001808900000804400100c9800580890009f
:1039100009005000200c98008200370070c6b300e8
:10392000804f55000300320070c4b300804f550033
:1039300014003a0058089000808f540004003d00a5
:10394000081090000038a30001003a00590c9800bc
:10395000580890000000e900500c980002003b005d
:103960000000eb00500c980070c6b300804f55006b
:1039700002003a005ac6b3000b0037005ac4b30025
:103980000900370010c6b300804f550002003a000e
:103990000ac7b3000400370010c4b300804f5500bd
:1039a00001003a000ac5b3001809900068009000b1
:1039b0003c7079008201e800130c98000c0278003a
:1039c000580890000000e00003003c000810900040
:1039d0000038a30017003200e8009000e0c2b300f6
:1039e00080f079008280e800110c9800580890005f
:1039f0000000e0000f0034008904e900890f500046
:103a000001003d00800478006800900000804000c4
:103a10000901780084007800eef307001808900090
:103a200000804400100c98005808900009005000d5
:103a3000200c980068009000980890000100400059
:103a40000086e8000a587800800078000d00e00049
:103a500004003500b0c2b300804878008c047800c0
:103a600004003700d0c2b300804878008c0478008e
:103a70008d06ea008005eb000a003700a200200056
:103a80008d00780070805700c50107000fb89700bf
:103a90009fb897007a81550001f17f008b05e800ff
:103aa000800678000d00e000f4ff3c00e18f550037
:103ab00009003c0050c6b300804f5500030032009f
:103ac00050c4b300804f550003003a0000c3b30058
:103ad000005e78008c0478000b00e00004003200e7
:103ae0000b00e900fa805700008040000600370014
:103af00000c3b300805c7800050037008b05e90047
:103b000002c3b300a05c41000b00e000fbff3c00df
:103b10006800900098089000010040000080540068
:103b2000300c98000810900074006000f00f5000f6
:103b30000e003a00780090009808900001004000c4
:103b4000a808900001004000b80890000100400063
:103b5000c80890008100400078089000808f5000d5
:103b600002003d0001005000000c98004f06be000e
:103b70004f05be004f04be000080fa0000000600a2
:103b80000200fa00889fbe008a9fbe008c1f78004a
:103b90008005780001057800020678000100e00049
:103ba00001003a006c8557000b04780001003700d3
:103bb0000804e800984478000900fb0066f3070059
:103bc0000000e000faff3a00d0c2b30080cf5400fa
:103bd0000500320000c0e90080cf5400020032002e
:103be00080447800010037000804e8000c017800e8
:103bf0008a007800080078003b0007000203be003e
:103c00000002be009a0f540001003a000b0d78002c
:103c10009a8f550005003a00e00f5200e08f5a00dd
:103c2000e00f5b00e08f5b0014003a00b0c2b3000d
:103c300080cf540006003a00e00f5200e08f5a0097
:103c4000e00f5b00e08f5b0020003d000b003700c1
:103c5000d0c2b30080cf54001c003a006000b8000e
:103c600002002000030028000020e10001a8e1007c
:103c700002b0e10003b8e1000e003600200220008f
:103c8000400889006b40400080cf540004003a0097
:103c90006000b80002002000030028000d0037007b
:103ca000f0ff2f00f1ff2f00f2ff2f00f3ff27009e
:103cb000080037006000b8006011b800040250002e
:103cc0008582580006035900878359000400be000e
:103cd0000601be004f0678004f05be004f04be002f
:103ce0000080fa0000000600fc874700889fbe00a5
:103cf0008a9fbe008c9fbe008e1f78000007780050
:103d00008106780082047800000478000100370002
:103d10000804e800184678000c00fb000ef30700ca
:103d20000000e000faff3a00d0c2b300804f560016
:103d30000500320000c0e900804f5600020032004a
:103d400000467800010037000804e8000900e000a0
:103d500005003500e18f54000300320040022000ce
:103d6000808f5400040034000d00e000b0003200e9
:103d70008e0e7800ae0037000900e0000e0034001f
:103d8000f08f54001a003a0000c3b300984f10009f
:103d900016003a009840900080c7b30080cf5000d2
:103da0000300320080c5b30080cf50000f003a00fe
:103db0000884e8000e003700a900200000c3b3000b
:103dc000984f10000a003a009840900080c7b30056
:103dd00080cf5000040032008900200080c5b3006d
:103de00080cf500002003a000884e800090120005a
:103df0000805780000c3b300010037000a05e80099
:103e00009a4f1000fdff32008a0578006022b8004a
:103e10006033b8002600370090ff210080c05000ba
:103e200081ef9f0009027800cfa2de000503780031
:103e3000860378000fb097009fb097002fb19700ce
:103e4000bfb19700a2030700d0b79f00e1b79f0062
:103e5000f2b79f0083bf9f000fe897000002fb00ae
:103e6000cfa2de0005037800860378008b05e8000a
:103e70000fb097009fb097002fb19700bfb1970088
:103e8000c0af9f00d1af9f00e2af9f00f3af9f0094
:103e90005fb09700efb097007fb197008fb99700a0
:103ea0000002420081824a0002034b0083834b00e0
:103eb00084b79f0095b79f00a6b79f00b7b79f0034
:103ec0001b00fb00acf207008000780009017800bd
:103ed00090ff2100aff20700800078000000e000b2
:103ee000cdff3a008b0f54000a003a000d00e000ad
:103ef0004f0032008e0e78006022b8006033b800a8
:103f000084b79f0095b79f00a6b79f00b7b79f00e3
:103f10004d0037008a80550040fd210060c07c00c4
:103f20000000fb00008050002c0033004240a9003c
:103f300020003c008fea97000500fb00cf80de00e8
:103f400001017800820178000fb297009fb29700bc
:103f50002fb39700bfb397000000520081805a0032
:103f600002015b0083815b000020e10001a8e10009
:103f700002b0e10003b8e1000e0039000902780048
:103f8000cfa2de000503780086037800bf02070099
:103f90004faa9700dfaa97006fab9700ffab97007f
:103fa0000400e1000588e1000690e1000798e100c7
:103fb0000a0032002002200040088900f0ff2f0094
:103fc000f1ff2f000001be0080b79f0091b79f0056
:103fd000a2b79f00b3b79f0011003700d0c2b30053
:103fe000804f56000e003a006000b8006011b80023
:103ff0000fb297009fb297002fb39700bfb39700ff
:104000000402500085825800060359008783590036
:1040100084b79f0095b79f00a6b79f00b7b79f00d2
:104020000d00e000080032008b0e7800060037001b
:104030006000b8006011b80080b79f0091b79f0082
:10404000a2b79f00b3b79f000fb097009fb0970033
:104050002fb19700bfb197004f0778004f06be0001
:104060004f05be004f04be00cf01b10000000600a6
:1040700000017800e60140001300780001002800ec
:10408000810360006f0060008009780012003a0030
:10409000220090000000e0000f003a0012009000a3
:1040a0000000e0000c003a00160020001200e000c2
:1040b0003800320008003700e40041009109780020
:1040c0000280e80090087800120878000009eb00f0
:1040d0007003530001003700160020001300e000b9
:1040e000f5ff3200e40241000282e80011003700cf
:1040f00080004000150078004f00de0080897000cd
:104100009500780081804000140078004f00de00a8
:10411000808a70009400780081804000120078004e
:104120004f00de00008a7000120078000009400095
:104130000603e90013007800ef0f5000ecff360093
:104140008282e800640241000e0037009200d10034
:10415000150078004f00dd00008970009500d10047
:10416000140078004f00dd00808a70009400d100b8
:10417000130078004f00dd00008a70009309d10021
:104180000603e80013007800ff0f5000efff3e0029
:10419000ef096000938973000600780000000600b4
:1041a00002027800809fbe00110009008200d80042
:1041b000000178004f00be0002a2b90084805000c8
:1041c000110098000208780000000600020ab900f9
:1041d000001bb9000200b8008100420081004300ca
:1041e00000000600889fbe008a9fbe00010578007f
:1041f0000100e0000400350008003c000000e00081
:10420000200032000500370060001000e080180038
:1042100002003b0001f02c001a0037000004be0031
:104220006011b8006b0920000982cf00020039003c
:104230000882cf000441b000694252000e003200f3
:1042400008003b0082817100610164008904d10093
:104250000884d3008b05e8000442e800f9ff3a0027
:10426000050037000804440089844c008b05e900f0
:104270000442e900fbff3a00db0007000af0a70058
:1042800001f0a0004f05be004f04be000000060074
:1042900003f0a200889fbe008a9fbe008c1f78009a
:1042a000f7000700fe0033006450e1004f003200c9
:1042b0006420e1005200320003826c0007003b00e2
:1042c0000905d0000306d000820f54000c065d00e3
:1042d00002003900020032008901780003067800ec
:1042e0008582550004003d000003fd008103fd00b0
:1042f0008502ea008b854200840f720002003b00b9
:1043000060001000e08018006011b8000005eb00ac
:104310007a28e1000a00390006007800c75ddd0058
:10432000f707b200878075002d0037008281710089
:104330000a017800610560008180d1000080d3000f
:104340008502e900f9ff3b0006044000878448002d
:1043500002003b0060041400e0841c000988a300f4
:10436000070032008a81710082817100610164005e
:104370008904d1000884d3008b05e80017003700ba
:104380000978a30013003a000b00e000130034008a
:104390008b05e9000804440089844c000a44740039
:1043a0000978a3000d003a000b00e000070034007c
:1043b0008b05e9000804440089844c0001003a00a0
:1043c0000b0020000978a300f7ff32000001eb008a
:1043d00002003700828171000a0178008200070024
:1043e0000cf0a70001f0a000b60037006420e10047
:1043f00002003a00838f6c00b60033000801be0053
:104400000200be00af003700889fbe008a9fbe003a
:104410008c1f78009a000700a100330003866c000f
:104420006450e1002e0032006420e10033003200cd
:104430006150e1002f0032006120e10031003200c4
:1044400085855500eb07b000090020000804200016
:10445000050037000804440089844c000a0031003c
:104460000603430087834b000001530081815b00fa
:10447000f8ff33000203be000800a0000804440057
:1044800089844c00f6ff3900c639dd0083017300d2
:1044900001003200130020008904d1000884d300f9
:1044a0000998a300050032000800a7000300a0003f
:1044b0008904d1000884d3008b05e8008904d10069
:1044c0000884d3000001eb000281d20046000700ff
:1044d00001f0a1000cf0a70001f0a0007900370066
:1044e0006420e1007b0032000801be000200be0033
:1044f000f7ff37006120e100760032006000b8006d
:10450000f3ff37000000200001f82700f0ff37001c
:104510001400200072003700889fbe008a9fbe00f2
:104520008c1f7800560007005d00330003866c0086
:104530006450e100240032006420e10027003200d2
:104540006150e100220032006120e10021003200d0
:104550008b854200eb07b1000134b800003ab80087
:104560000804420089844a00013ab8000030b800cb
:104570008880400009014a00040033000000400028
:1045800081804800020149008b05e900c909dd006e
:10459000830170000100320013002000c814de0007
:1045a0004814dd004709de001200b200c808de0032
:1045b000088470000c00070001f0a1000cf0a700b7
:1045c00001f0a0003f0037006120e100410032000f
:1045d0000801be000200be00f7ff37006150e10095
:1045e000fcff3a003b00370081002000618055004d
:1045f0000b003d000b00200061fe2f000100e100d8
:104600001d00340082817100610164008904d100c1
:104610000884d3000000e800faff3a00710020008f
:1046200061006400030070000200600009003200b5
:1046300061044400e0844c000988a50005003200b4
:104640008b05e8006808e10002003a008904d10007
:104650000884d300f20f20000258e10005003d005d
:10466000c75ddd00f907b200898075000800780099
:10467000000006000bf827008b0078000000050002
:104680000004be00310007000003be000405be00a8
:104690000200be002d000700844f750000000600d8
:1046a0000200be006450e100050036006420e10015
:1046b000020036000968a30001003a000800be00ad
:1046c0000160a0004f0678004f05be004f04be00f9
:1046d00000000600f0ff2f00f1ff2700f9ff370070
:1046e000889fbe008a9fbe00841f7800e4ff0700f9
:1046f0004f00780011003300f0ff2f00838f6c0013
:1047000006003b00040565000a00a700080037000a
:1047100009f0a6001000200008003700820f5400a6
:10472000838f5c00030039001000200001003e0070
:104730000000200009f0a7000000ea004f05be00bd
:104740004f04be000000e00000000600c70ade00c3
:10475000f107b200f50fb20008003200e1cf4200cd
:10476000020032000170a00024000500810f7000db
:10477000010032000408050044000500810f7000ac
:1047800002003a00140005008502e9000000400024
:1047900081c04800fcff3b000170a0002400050020
:1047a0006022b800060220000000d0008180d20004
:1047b0000482d2008582d2000000a00002025200d2
:1047c00083825a00030031000202420083824a00c1
:1047d0000000a1000603e900f3ff3a000000060014
:1047e00081037800d9ff07000001be006000b80017
:1047f0000478a30013003a006220e10015003e0097
:104800000d0039008301d1000281d3008180d300e3
:104810008301d1000281d3008180d3008301d100c4
:104820000281d3008180d3000538b000c42add00a6
:10483000f300b2008381720007f0a70003f0a0002c
:1048400000000600f3ff2700f2ff2f006110b900ff
:10485000fbff370003ff2700f7ff3700d0ff0700fb
:104860000400be0000000600839f68000100e00015
:1048700002003d0060001000e08018000300e0002e
:1048800002003d0060011100e0811900c4ff070033
:104890004f00e00002003b0060001000e0801800c4
:1048a00000000600881f7800000478005001be0058
:1048b0004000be0004004000858048000601490019
:1048c00087814900009cbe000294be000400e10004
:1048d0000588e1000690e1000798e1000200310040
:1048e000680044001008e8004f047800000006004b
:1048f000f4874700889fbe008a9fbe008c9fbe0041
:104900008e1f78000205be000004be00d4b79f00d1
:10491000e5b79f00f6b79f0087bf9f000000eb0040
:10492000c0b79f00b0b79f00a0b79f0090b79f008f
:1049300080b79f000d042000bfb097004fb09700d4
:10494000000140000000e0000f003d004f08de00c5
:1049500000007100c0b79f009e00070001003d00ed
:1049600012002000a100070001003d0012002000fd
:10497000a6000700b1000700b60007000f004000c6
:10498000c8ff0700220037004f08de000006710054
:10499000ccb79f008f00070001003d0012002000ef
:1049a0009200070001003d00120020009700070060
:1049b000a20007000fb297009fb297002fb3970095
:1049c000bfb39700a90007000000520081805a0081
:1049d00002015b0083815b0080b79f0091b79f005d
:1049e000a2b79f00b3b79f000007eb009f0007002e
:1049f0000020e10001a8e10002b0e10003b8e100fd
:104a0000010031001e0020000e005600c0b79f00bc
:104a10004fb297000400e0000700350010002000ae
:104a2000010020006011b800080470008984700043
:104a30000a0571008b8571008d06e900beff3a0002
:104a40000400e00003003d00820007000f0040006a
:104a500094ff07004fa897000000e00004003a0010
:104a60000fb497009fb497002fb59700bfb597007c
:104a7000940007004f0778004f06be004f05be00a8
:104a80004f04be004f01b10000000600881f7800ef
:104a900018002000881f780095ff07008f87e90025
:104aa0004f04780000000600801feb0090ff070015
:104ab0008f87e90000000600889fbe008a9fbe0025
:104ac0008c1f78006e00070007003d007300070090
:104ad000e00f5b00e08f5b0007003d003200070045
:104ae0000006eb00040037003400070002003d0020
:104af0002a0007001c00200072000700e3ff0700e7
:104b00000203be000002be000c00e0000100320003
:104b1000220007000400be000601be004f06780018
:104b20004f05be004f04be0000000600889fbe0077
:104b30008a9fbe008c1f78005100070005003d00d1
:104b400056000700e00f5b00e08f5b0006003d00b1
:104b5000040037001900070003003d006000b800a2
:104b60006011b8001000070056000700ceff0700d4
:104b70000203be000002be000c00e0000100320093
:104b8000060007000400be000601be004f067800c4
:104b90004f05be004f04be00000006006000b800d4
:104ba0006011b800000037000402500085825800f0
:104bb0000603590087835900000006000006eb0039
:104bc000e00f5200e08f5a00e00f5b00e08f5b00c7
:104bd000000006000180400090b79f000001eb003c
:104be0008fb097000100e000000006000200700096
:104bf00090b79f000180400080b79f000001eb004c
:104c0000ffa897000100e00000000600020070000d
:104c100080b79f00018040006faa9700cf20de0080
:104c200001007000f0af9f00040242002500070061
:104c30004f18de000002720000000600e4af9f0083
:104c40000804440089844c000a054d008b854d0002
:104c5000000006003fb29700cfb297005fb3970005
:104c6000efb3970000fe2f00000006003fb0970052
:104c7000cfb097005fb19700efb19700000006003a
:104c80000205be000004be00e00f5000e08f580097
:104c9000e00f5900e08f5900000006006000b800e6
:104ca0006011b80008045000898458000a055900b2
:104cb0008b8559001c002000e00f5200e08f5a0045
:104cc000000006000800be000a01be000000060049
:104cd000889fbe008a9fbe008c1f78000205be0020
:104ce0000004be000006eb00e00f5000e08f58000b
:104cf000e00f5900e08f590007003d006000b80048
:104d00006011b80008045000898458000a05590051
:104d10008b8559001c002000e00f5200e08f5a00e4
:104d2000e00f5b00e08f5b0002003d000f0007001a
:104d30000c00a2000800be000a01be001c01070012
:104d40000203be000002be000c00e00001003200c1
:104d5000060007000400be000601be004f067800f2
:104d60004f05be004f04be00000006006000b80002
:104d70006011b800040250008582580006035900f3
:104d800087835900000006008f1fd1002a01070009
:104d90008f87e9000000e000000006001400fa0020
:104da000889fbe008a9fbe008c9fbe000004be008c
:104db0000205be00680047000a90be000890be00d1
:104dc000460107000070a7000bf0a100304320004f
:104dd0009e02900080825200b0fe2f000028e10069
:104de00011003d00b0fc2f000028e1001500340048
:104df0001e0990008e0890007e0090000501b00012
:104e00000201d1008180d3000080d3008502e80038
:104e1000fbff3a000b00e0006b013b00600010005c
:104e2000e080180068013700f0ff2f00f1ff270035
:104e30000b00e00064013b0001002800000020009e
:104e4000610137006000b8005f0137004f89de0064
:104e5000820178006101370007f0a2009601370057
:104e6000809feb00f40007008f87e9000000e0005e
:104e7000000006002800fa00889fbe008a9fbe003e
:104e80008c9fbe0003866b003b0107000028a30037
:104e900064003a000128a30067003a000008a3005c
:104ea00062003a000108a30065003a001e0090006d
:104eb000be08900081064000ed3fb100f48057002d
:104ec000ee019000111ab8008e099000311bb80055
:104ed0009e099000311cb800511db800f4855700a0
:104ee00046000700fe0190003a0007008b85e800ad
:104ef0003e0007008e09900040000700ee01900080
:104f0000340007008b85e800380007008e09900008
:104f1000400007009e0990001b18b800890440005b
:104f20000a854800fe019000340007008b85e800e8
:104f300038000700ee019000300007008e09900055
:104f40001b18b800890440000a8548000a98a3008d
:104f500008003a000402420085824a0006034b0022
:104f600087834b0008044c0089844c000a054d00df
:104f70008d06e90084827200850273004c3add00e0
:104f8000850272000100320015002000443ade0064
:104f90001400b2004538de00cb45dd000b00700088
:104fa000c540de00cb4ddd008b8070004549de0042
:104fb000cb55dd000b017100c551de000d037800fb
:104fc000ba01070003f0a1000cf0a70003f0a00055
:104fd000fd0037001b18b80085024000068348001a
:104fe000e0834b0060044c00070037001b18b8003a
:104ff0000603400087834800faff37001b18b800fb
:105000008703400008844800e0844c0060054d00a0
:10501000000006001b18b8000804400089844800fe
:10502000faff37000108a300e4003a005800be0070
:105030005801be00e3ff37000008a300df003a007c
:1050400009047800f9ff37002800fa00889fbe00a5
:105050008a9fbe008c9fbe0003866b00c6000700bf
:105060006400e100440032006408e1004a003200bc
:105070006100e100460032006108e10049003200b1
:10508000ec0647006000b8003d02be003d03be00d4
:10509000f48657006011b8003d04be003d05be0017
:1050a0007d0320000b0037000000a0008d06e90002
:1050b000130032000402420085824a0006034b00be
:1050c00087834b00000040008180480002014900b6
:1050d000838149000802520089825a000a035b005a
:1050e0008b835b00f0ff3b000802420089824a008c
:1050f0000a034b008b834b008d06e900edff3a005d
:105100008482720086827200f707b2008782720082
:1051100001003200150020001e0490003e0b90009c
:1051200006035400e63fb0000368a3000700320006
:105130000000a7000500a0008301d1000281d30078
:105140008180d3000080d3000603e8008301d100f2
:105150000281d3008180d3000080d3000002eb00e5
:105160000482d2005101070003f0a1000cf0a70057
:1051700003f0a00094003700640247006408e100d7
:105180008e0032003400be003401be00f6ff37004e
:105190006108e100890032006011b8006000b800c9
:1051a000f1ff370003ff270002002000fbff37005c
:1051b000889fbe008a9fbe008c9fbe000404b8007a
:1051c0000506b8008904460060854e000606b80052
:1051d0000a054600e0854e000706b8008b0546002c
:1051e000040eb800890446000a854e00e0854d0093
:1051f000050eb8000a0546008b854e00060eb80065
:105200008b0546000416b8000a0546008b854e0043
:105210000516b8008b054600041eb8008b05460035
:105220000800be000a01be004f06be004f05be00ca
:105230004f04be0000000600889fbe008a9fbe008b
:105240008c9fbe000404be000605be00809fbe0009
:10525000829fbe0041010700040678000800be00de
:105260000a01be003d010700840678004f03be001e
:105270004f02be008d4f76007fb0970013003300c1
:10528000f0ff2f008b8f6b0006003b000d066600c1
:105290000c00a7000a00370007f0a600100020004d
:1052a0000a003700880f5200898f5a008a0f5b006e
:1052b0008b8f5b00030039001000200001003e00ce
:1052c0000000200007f0a7000000ea004f06be0023
:1052d0004f05be004f04be000000060080007800ad
:1052e0005002be005003be004439de00f700b20099
:1052f000f37f200003016100090032000218e10081
:1053000016003a00850172008301730083817300e7
:105310000008200015003a0040002000130037006c
:1053200085017200830173008381730005003a00d8
:1053300004a8be0006a8be00100020000b00370025
:105340000201e9000402420085824a0006034b0084
:1053500087834b000748a300f9ff32000740a000f5
:1053600004a8be0006a8be0020002000800098000f
:105370009200980000000600680447000294be00f6
:105380000094be00fc0447008694be008494be00d6
:1053900009007800d1ff070008007800cfff070060
:1053a00099007800814f70000b003b000800be00a0
:1053b000fc0007004f00b10003003700f3ff270097
:1053c000f2ff2f006110b9004f06be004f05be006e
:1053d0004f04be000080fa0000000600889fbe0057
:1053e000830478000300e0002c00350003003c003b
:1053f0000082700004027100260032003643200053
:10540000c50020008383cf000a0039000541b100a8
:105410008283cf00070039000541b1008183cf00ae
:10542000040039000541b1008083cf00010039003c
:105430000541b10085c353006022b800120032005c
:105440000a003b0084827200610260008301d10087
:105450000281d3008180d3000080d3000603e800de
:105460008743e800f7ff3a000700370000004000dc
:105470008180480002014900838149000603e90058
:105480008743e900f9ff3a008800070009f0a70008
:1054900003f0a0004f04be000000060060001000f2
:1054a000e080180060011900e0811900d3ff3b0083
:1054b000033e2c00f7ff37002800fa00889fbe004b
:1054c0008a9fbe008c9fbe00070678008786690011
:1054d0000c003b00030478008704780008f0a1006a
:1054e00009f0a100840f5000858f5800860f5900e5
:1054f000890f5c00030033000cf0a20001003a00a9
:105500000cf0a1009cff07006400e1005f00320086
:10551000780147006408e100610032006c01470037
:10552000748557003200be001201be003a04be006e
:105530001a05be001e039000be0a900085035300aa
:1055400006003d000004fd008104fd000205fd0091
:105550008305fd008703ea00050378000df8a3002a
:105560000400320060041400e0841c0060051d008b
:10557000e0851d006022b8007d0320000d38e100a9
:105580008006eb000b0039004433dd00f300b2006d
:105590008301730039003700848272000d027800a5
:1055a000e10664008b85d1000a85d3008984d3008d
:1055b0000884d3008703e900f7ff3b0008004000a0
:1055c000898048000a0149008b81490004003b00a2
:1055d00060001000e080180060011900e0811900ef
:1055e0000358a300090032008d8272008482720089
:1055f000610260008301d1000281d3008180d30069
:105600000080d3000603e8001b0037000348a30016
:1056100017003a000600e000170034000603e90016
:105620000d00a300000048008180480002014900ed
:10563000838149000348a3000f003a000600e00000
:10564000090034000603e9000000400081804800a2
:10565000020149008381490001003a000003eb0088
:105660000348a300f5ff32006022b80002003700b3
:1056700084827200618266000c00070003f0a100c2
:105680000cf0a70003f0a0004fff370064014700b3
:105690006408e10002003a000df8a30047ff3a0059
:1056a0003200be001201be0047ff37001800200084
:1056b00057002000080453000d003d0006002000a4
:1056c00097fc2f000740e1001e0034008482720026
:1056d000610260008301d1000281d3008180d30088
:1056e0000080d3000804e800f8ff3a0047002000db
:1056f0006104600005047400040464000d003200bd
:1057000061004000e080480060014900e0814900fc
:1057100003b8a500070032000603e8006538e10081
:1057200004003a008301d1000281d3008180d300bc
:105730000080d300f87f20000830e100030035002e
:10574000080378006000b8006011b8004433dd0041
:10575000f300b200830173000000060005ff27007c
:1057600005826100070032000428e10001003200d8
:10577000240005000600070001003a00440005006f
:105780000408050002000700f9ff3a0014000500b4
:105790006f826100810270008502710085027200d3
:1057a00000000600e48240001078a30007003200e9
:1057b000640240001178a3003400be001401be0052
:1057c000040032000330a700000006003500be00d0
:0c57d0001501be000330a0000000060020
:020000040000fa
:020000040001f9
:0457f0003fff000077
:020000040000fa
:020000040001f9
:0457f400c21c0000d3
:020000040000fa
:020000040001f9
:0457f800bdfa0000f6
:020000040000fa
:020000040001f9
:0457fc007f3f0000eb
:020000040000fa
:10000800be540000be540000be540000be540000a0
:10001800be540000be540000be540000be54000090
:10002800be540000be540000be540000be54000080
:10003800be540000be540000be540000ec50000046
:10004800be540000be540000be5400009449000095
:100058007c490000be540000be540000be5400009d
:10006800be540000be540000be540000be54000040
:10007800be540000be540000be540000be54000030
:10008800be540000be540000be540000be54000020
:10009800be540000be540000be540000be54000010
:1000a800be540000be540000be540000be54000000
:1000b800be540000be540000be540000be540000f0
:1000c800be540000be540000be540000be540000e0
:1000d800be540000be540000be540000be540000d0
:1000e800be540000be540000be540000be540000c0
:1000f800be540000be540000be540000be540000b0
:10010800be540000be540000be540000be5400009f
:10011800be540000be540000be540000be5400008f
:10012800be540000be540000be540000be5400007f
:10013800be540000be540000be540000be5400006f
:10014800be540000be540000be540000be5400005f
:10015800be540000be540000be540000be5400004f
:10016800be540000be540000be540000be5400003f
:10017800be540000be540000be540000be5400002f
:10018800be540000be540000be540000be5400001f
:10019800be540000be540000be540000be5400000f
:1001a800be540000be540000be540000be540000ff
:1001b800be540000be540000be540000be540000ef
:1001c800be540000be540000be540000be540000df
:1001d800be540000be540000be540000be540000cf
:1001e800be540000be540000be540000be540000bf
:0801f800be540000be540000db
:020000040000fa
:10020800be540000be540000be540000be5400009e
:10021800be540000be540000be540000be5400008e
:10022800be540000be540000be540000be5400007e
:10023800be540000be540000be540000ec50000044
:10024800be540000be540000be5400009449000093
:100258007c490000be540000be540000be5400009b
:10026800be540000be540000be540000be5400003e
:10027800be540000be540000be540000be5400002e
:10028800be540000be540000be540000be5400001e
:10029800be540000be540000be540000be5400000e
:1002a800be540000be540000be540000be540000fe
:1002b800be540000be540000be540000be540000ee
:1002c800be540000be540000be540000be540000de
:1002d800be540000be540000be540000be540000ce
:1002e800be540000be540000be540000be540000be
:1002f800be540000be540000be540000be540000ae
:10030800be540000be540000be540000be5400009d
:10031800be540000be540000be540000be5400008d
:10032800be540000be540000be540000be5400007d
:10033800be540000be540000be540000be5400006d
:10034800be540000be540000be540000be5400005d
:10035800be540000be540000be540000be5400004d
:10036800be540000be540000be540000be5400003d
:10037800be540000be540000be540000be5400002d
:10038800be540000be540000be540000be5400001d
:10039800be540000be540000be540000be5400000d
:1003a800be540000be540000be540000be540000fd
:1003b800be540000be540000be540000be540000ed
:1003c800be540000be540000be540000be540000dd
:1003d800be540000be540000be540000be540000cd
:1003e800be540000be540000be540000be540000bd
:0803f800be540000be540000d9
:020000040000fa
:1057dc004d4500004f5700000d0a0000004200002c
:1057ec0049540000202500006420000049530000ab
:1057fc0020480000490d00000a000000424900004a
:10580c0054200000256400002049000053200000b3
:10581c004c4f00000d0a00000044000041540000f1
:10582c00453a0000200000000d0a00000054000062
:10583c00494d0000453a000020000000426f000076
:10584c00617200006420000041640000647200007a
:10585c0065730000732000006973000020250000b0
:10586c00642000000d0a0000004200006f6100007f
:10587c007264000020540000797000006520000064
:10588c006973000020250000642000000d0a000050
:10589c0000540000656d000070200000536500008e
:1058ac006e7300006f720000205b00004a3600002f
:1058bc005d200000697300002025000066200000b8
:1058cc00646500006772000065650000730d0000e0
:1058dc000a000000546500006d70000020530000a9
:1058ec00656e0000736f0000722000005b4a0000c0
:1058fc00375d000020690000732000002566000061
:10590c00206400006567000072650000657300008c
:10591c000d0a000000540000656d000070200000ae
:10592c00536500006e7300006f720000205b000076
:10593c004a3800005d20000069730000202500003b
:10594c006620000064650000677200006565000059
:10595c00730d00000a000000546500006d7000001b
:10596c0020530000656e0000736f00007220000071
:10597c005b4a0000395d00002069000073200000c4
:10598c002566000020640000656700007265000059
:10599c00657300000d0a000000540000656d0000e6
:1059ac0070200000536500006e7300006f720000e1
:1059bc00205b00004a310000335d000020690000cc
:1059cc00732000002566000020640000656700005d
:1059dc0072650000657300000d0a000000540000a1
:1059ec00656d000070200000536500006e730000b0
:1059fc006f720000205b00004a310000355d000032
:105a0c00206900007320000025660000206400005f
:105a1c006567000072650000657300000d0a0000e8
:105a2c0000540000656d00007020000053650000fc
:105a3c006e7300006f720000205b00004a310000a2
:105a4c00365d000020690000732000002566000010
:105a5c00206400006567000072650000657300003b
:105a6c000d0a000000540000656d0000702000005d
:105a7c00536500006e7300006f720000205b000025
:105a8c004a310000375d00002069000073200000df
:105a9c002566000020640000656700007265000048
:105aac00657300000d0a0000000d00000a52000092
:105abc0065740000757200006e65000064200000c3
:105acc00566100006c750000652000003d20000050
:105adc00256600000d0a000000540000494d00002e
:105aec00452000005345000054200000464f0000a4
:105afc00524d0000415400003a200000686800003c
:105b0c003a6d00006d3a0000737300003a770000a4
:105b1c00643a0000444400003a4d00004d3a000045
:105b2c00595900000d0a000000770000642800009d
:105b3c0077650000656b000020640000617900004f
:105b4c00293a000020300000203d000020530000c6
:105b5c00756e000064610000792c0000203100009b
:105b6c00203d0000204d00006f6e000064610000bd
:105b7c00792c000020650000746300002e0d0000dd
:105b8c000a00000025680000686400003a25000047
:105b9c0068680000643a0000256800006864000032
:105bac003a25000068680000643a0000256800008f
:105bbc00686400003a25000068680000643a000040
:105bcc002568000068640000004500005252000087
:105bdc003a20000046410000494c000045440000ba
:105bec00205400004f2000005345000054200000ba
:105bfc0052540000430d00000a0000000000000099
:105c0c000000000000000000000000000000000088
:105c1c000000000000000000000000000000000078
:105c2c000000000000000000000000000000000068
:105c3c000000000000000000000000000000000058
:105c4c000000000000000000000000000000000048
:105c5c000000000000000000000000000000000038
:105c6c000000000000000000000000000000000028
:105c7c000000000000000000000000000000000018
:105c8c000000000000000000000000000000000008
:105c9c0000000000000000000000000000000000f8
:105cac0000000000000000000000000000000000e8
:105cbc0000000000000000000000000000000000d8
:105ccc0000000000000000000000000000000000c8
:105cdc0000000000000000000000000000000000b8
:105cec0000000000000000000000000000000000a8
:105cfc000000000000000000000000000000000098
:105d0c000000000000000000000000000000000087
:105d1c000000000000000000000000000000000077
:105d2c000000000000000000000000000000000067
:105d3c00000000000000000000000000537500008f
:105d4c006e640000617900002c200000004d000002
:105d5c006f6e000064610000792c000020000000d0
:105d6c00547500006573000064610000792c00001c
:105d7c002000000057650000646e00006573000091
:105d8c0064610000792c00002000000054680000c1
:105d9c007572000073640000617900002c20000013
:105dac00004600007269000064610000792c00005c
:105dbc002000000053610000747500007264000044
:105dcc00617900002c200000005b00003f3f0000c8
:105ddc003f5d000064610000792c00002000000091
:105dec004a6100006e7500006172000079200000ad
:105dfc0000460000656200007275000061720000d0
:105e0c0079200000004d0000617200006368000002
:105e1c002000000041700000726900006c2000003e
:105e2c00004d000061790000200000004a75000060
:105e3c006e650000200000004a7500006c790000bf
:105e4c0020000000417500006775000073740000ad
:105e5c00200000005365000070740000656d0000a8
:105e6c006265000072200000004f000063740000a7
:105e7c006f62000065720000200000004e6f000091
:105e8c00766500006d620000657200002000000065
:105e9c0044650000636500006d62000065720000df
:105eac00200000005b3f00003f3f00005d6d0000e4
:105ebc006f6e0000746800002000000025300000a8
:105ecc00326400002c20000000320000302500005d
:105edc003032000064000000253000003264000005
:105eec003a25000030320000643a000025300000f2
:105efc003264000000000000474500005400000020
:105f0c005345000054000000434c00004541000084
:105f1c00527c0000434c0000520000004845000039
:105f2c004c4c00004f2000004b4900005454000022
:105f3c00590000000000000082af0000e0300000bb
:105f4c0086af0000f03000008aaf00000031000086
:105f5c0094af000010310000a0af00000000000062
:105f6c00444900004e000000444f0000555400000e
:105f7c0000540000494d0000450000004244000060
:105f8c005f4100004444000000420000445f0000f8
:105f9c0054590000504500000041000044430000eb
:105fac0000540000454d000050000000b6af00004a
:105fbc0020310000baaf000060310000bfaf00001c
:105fcc00a0310000c4af0000de310000cbaf0000f8
:105fdc0010320000d3af000096330000d7af0000a2
:105fec0042320000a0af000000000000435300004c
:105ffc005f41000044440000004900004e54000082
:10600c00005000004f54000030000000504f0000c2
:10601c0054310000005000004f5400005f5200004b
:10602c0053000000baaf000020350000bfaf0000e5
:10603c003a350000fcaf00009435000003b00000be
:10604c00ac35000007b00000d23500000cb00000e9
:10605c00ec35000011b0000006360000a0af0000c7
:10606c0000000000baaf00001e360000a0af000018
:10607c0000000000313300003a320000313a0000d9
:10608c003533000000530000657000002020000034
:10609c00312000003230000031310000000d0000d2
:1060ac000a4600004f430000452000004348000012
:1060bc00415300005349000053200000454e00009e
:1060cc0056490000524f00004e4d0000454e000056
:1060dc00544100004c200000424f0000415200008f
:1060ec004420000042750000696c00007420000020
:1060fc006f6e00002025000073200000617400000a
:10610c0020250000730d00000a000000200900008b
:10611c0000450000525200002025000030340000e1
:10612c00640d00000a00000052440000590d0000ec
:10613c000a00000000000000000000000000000049
:10614c000000000000000000000000000000000043
:10615c000000000000000000000000000000000033
:10616c000000000000000000000000000000000023
:10617c000000000000000000000000000000000013
:10618c000000000000000000000000000000000003
:10619c00000000002009000000200000003000007a
:1061ac00313200003334000035360000373800003f
:0461bc0039000000a6
:020000040000fa
:1061c0000200fa00000f780052002000c1fd2a00f2
:1061d0001e007800180e07000080fa00000006007c
:1061e0000200fa00000f78005200200081012b000d
:1061f0001e007800100e07000080fa000000060064
:106200000200fa00000f78005200200081032b00ea
:106210001e007800080e07000080fa00000006004b
:106220000200fa00000f7800e1be2a0010002000f2
:10623000a50b07000000eb000080fa00000006003c
:106240000400fa0010079800a20020008000eb0074
:106250001e009000dce80700000f78001e007800a8
:106260007f0a07000000e000080032001e007800ee
:10627000801f780050bf2a00801f780000dd2100b9
:106280006be90700e4875700070037001e0078001d
:10629000801f780040c02a00801f780000dd2100a8
:1062a00063e90700e487570001dd210010002000aa
:1062b000850b07000000eb000080fa0000000600dc
:1062c0000400fa0010079800a20020008000eb00f4
:1062d0001e009000bce80700000f78001e00780048
:1062e000a90907000000e000080032001e00780045
:1062f000801f780050bf2a00801f780000dd210039
:106300004be90700e4875700070037001e007800bc
:10631000801f780040c02a00801f780000dd210027
:1063200043e90700e487570001dd21001000200049
:10633000650b07000000eb000080fa00000006007b
:106340000a00fa00400798000e007800b90607001e
:1063500001dd21000e0078006907070031c12a0025
:1063600010002000580b070001dd21001000200064
:10637000550b0700a1c12a0010002000520b070096
:1063800001dd21000e0078001b080700d1c12a00a2
:10639000100020004c0b070001dd21001000200040
:1063a000490b0700a1c12a0010002000460b07007e
:1063b0000000eb000080fa00000006000600fa0072
:1063c00020079800a20020008000eb002e00900023
:1063d0007de80700100798000000eb00000f780030
:1063e00010002000cc020700000f78001e0078008b
:1063f000801f780040c22a00801f780000dd210045
:106400000be90700e487570001dd210010002000a0
:106410002d0b07000000eb000080fa0000000600d2
:106420000600fa0020079800a20020008000eb0080
:106430002e00900064e80700100798000000eb00b1
:10644000000f780010002000df020700000f780026
:106450001e007800801f7800b0c32a00801f7800db
:1064600000dd2100f2e80700e487570001dd21008c
:1064700010002000140b07000000eb000080fa0061
:10648000000006000a00fa0030079800a200200071
:106490008000eb003e0090004be8070020079800ca
:1064a0006000b800008fbe002e00900040079800ea
:1064b000ce009000e38f50004a0032004e00900062
:1064c000e30f50000a003c00ce009000e18f500026
:1064d000240032004e009000e10f500031003c00db
:1064e000ce0090000100e0000e0032008c0037006a
:1064f0004e009000e50f50005a003200ce00900090
:10650000e58f5000470035004e009000e60f500028
:1065100064003200ce009000e78f5000710032001e
:106520007f00370002002c00934724000000eb009e
:1065300051050700008fbe001e00be00809fbe00f8
:10654000f0c42a00801f780000e12100b8e80700ad
:10655000e687570001e1210010002000da0a070059
:106560006f00370002002c00934724001000200029
:1065700041050700008fbe001e00be00809fbe00c8
:1065800000c72a00801f780000e12100a8e807006a
:10659000e687570001e1210010002000ca0a070029
:1065a0005f00370002002c009347240020002000e9
:1065b00031050700008fbe001e00be00809fbe0098
:1065c00010c92a00801f780000e1210098e8070028
:1065d000e687570001e1210010002000ba0a0700f9
:1065e0004f00370002002c009347240030002000a9
:1065f00021050700008fbe001e00be00809fbe0068
:1066000020cb2a00801f780000e1210088e80700e5
:10661000e687570001e1210010002000aa0a0700c8
:106620003f00370002002c00934724004000200068
:1066300011050700008fbe001e00be00809fbe0037
:1066400030cd2a00801f780000e1210078e80700a3
:10665000e687570001e12100100020009a0a070098
:106660002f00370002002c00934724005000200028
:1066700001050700008fbe001e00be00809fbe0007
:1066800050cf2a00801f780000e1210068e8070051
:10669000e687570001e12100100020008a0a070068
:1066a0001f00370002002c009347240060002000e8
:1066b000f1040700008fbe001e00be00809fbe00d8
:1066c00070d12a00801f780000e1210058e80700ff
:1066d000e687570001e12100100020007a0a070038
:1066e0000f00370002002c009347240070002000a8
:1066f000e1040700008fbe001e00be00809fbe00a8
:1067000090d32a00801f780000e1210048e80700ac
:10671000e687570001e12100100020006a0a070007
:106720000000eb000080fa00000006001e00fa00e6
:10673000300f9800a20020008000eb003e0890007f
:10674000a1e70700200f98000000eb00100f980051
:106750000000eb00000f98000000eb0070079800ad
:106760000000eb00600798000000eb005007980065
:106770000000eb00400798000000eb003007980095
:106780006000b80010079800210798000000eb0097
:10679000000f78002e089000e70f500039003c00f1
:1067a00080002000000f78002e089000500f980005
:1067b000de089000e38f5000230032005e08900056
:1067c000e30f50000a003c00de089000e18f50000b
:1067d000170032005e089000e10f500017003c00e7
:1067e000de0890000100e0000e003200900037004b
:1067f0005e089000e50f500019003200de0890009e
:10680000e58f5000130035005e089000e60f500041
:1068100016003200de089000e78f500016003200ac
:1068200083003700600820003007980035003700eb
:10683000600c20003007980032003700600920000b
:10684000300798002f003700600d200030079800b7
:106850002c003700600a200030079800290037001c
:10686000600e20003007980026003700600b2000e3
:106870003007980023003700600f20003007980091
:106880002000370090002000000f78002e089000b4
:10689000600f9800ee089000e98f50001100320060
:1068a0006e089000e90f500004003c00ee089000d4
:1068b000e88f5000080032005d0037006e0890003d
:1068c000ea0f50000a003200ee089000eb8f5000f3
:1068d0000a00320056003700600920003007980097
:1068e00008003700600a20003007980005003700d4
:1068f000600520003007980002003700600d20007e
:10690000300798008000eb001e0078006907070040
:1069100060c2a900200020007e0f070000000000d8
:106920003e0090007b0f07000000eb00790f07008e
:10693000100f98000000eb00760f0700000f980082
:106940000000eb00730f0700700798001100200093
:106950001e007800570707001e0890006007980087
:106960006e0090004800dd00600798008e089000df
:10697000f00f2000808060006e0090000100700029
:10698000600798006e0090000000400060079800cb
:106990007e0090004700de00700798000000eb00ca
:1069a000500798005e0090004800dd0050079800f6
:1069b000fe009000f00f2000808060005e009000dc
:1069c0000100700050079800ee0090005e009000fb
:1069d000008070004007980022002000ce00900048
:1069e0002e089000770a0700cf80de00fdf5070033
:1069f00010079800210798001e009000ae0090003c
:106a0000809fbe00b0d52a00801f780000e12100e1
:106a100087e70700e687570001e12100100020000a
:106a2000a90907000000eb00400f980001003700a3
:106a3000010037004e0890000080fa0000000600b8
:106a40000400fa0010079800a20020008000eb006c
:106a50001e009000dce60700000f78001100200007
:106a60001e007800130707000000eb000080fa000a
:106a7000000006000c00fa00400798004e0090004d
:106a8000104078000004e00009003a0031d72a00e5
:106a9000100020008c090700b1d92a001000200046
:106aa000890907000000eb00500798001b00370021
:106ab0008e1f78000e00e800801f78000e80e8002e
:106ac000801f780063004700801f78006600470041
:106ad000801f780065004700801f78006400470031
:106ae000801f780080dc2a00801f78004e00900014
:106af0006ce70700f08757000e0078004504070098
:106b00000000e00003003a00b1de2a00100020007f
:106b10006d0907000000eb00500798005e00900030
:106b20000080fa00000006000400fa001007980038
:106b3000a20020008000eb001e009000a2e60700eb
:106b4000000f78001e007800490007000000eb00ed
:106b50000080fa00000006000400fa001007980008
:106b6000a20020008000eb001e00900096e60700c7
:106b7000000f78001e00e00004003a008000eb00e7
:106b800050002000cb060700030037001100200052
:106b900050002000c70607000000eb000080fa004c
:106ba000000006000400fa0010079800a200200070
:106bb0008000eb001e00900083e60700000f7800c5
:106bc0009e0078000000eb00ca0307000000eb0005
:106bd0000080fa00000006000400fa001007980088
:106be000a20020008000eb001e00900076e6070067
:106bf000000f78009e00780010002000bd03070001
:106c00000000eb000080fa00000006000400fa001b
:106c100010079800a20020008000eb001e009000ea
:106c200069e60700000f780010002000ca03070083
:106c30000000eb000080fa00000006000400fa00eb
:106c400010079800a20020008000eb001e009000ba
:106c50005de60700000f78008000eb001e00780062
:106c6000940607000000eb000080fa000000060018
:106c70000600fa00000f78001e0078006101b900dc
:106c800012079800230798009000200001002000c0
:106c90001e019000ae019000800f5100818f5900bd
:106ca0008f003e001e009000ae00900000600100ca
:106cb0000900370015003700210037002d0037008c
:106cc0003900370045003700510037005d003700bc
:106cd00069003700750037008000eb000000eb0012
:106ce000740607008000eb0010002000710607000a
:106cf0008000eb00200020006e0607008000eb0003
:106d0000300020006b0607008100370011002000d2
:106d10000000eb00670607008000eb001000200079
:106d2000640607008000eb002000200061060700d9
:106d30008000eb00300020005e0607007400370082
:106d40008000eb000000eb005a0607001100200055
:106d500010002000570607008000eb0020002000f4
:106d6000540607008000eb003000200051060700a9
:106d700067003700110020000000eb004d060700ff
:106d800011002000100020004a0607008000eb00e0
:106d900020002000470607008000eb0030002000a4
:106da000440607005a0037008000eb000000eb00ab
:106db000400607008000eb00100020003d060700a1
:106dc00011002000200020003a0607008000eb00a0
:106dd00030002000370607004d003700110020006a
:106de0000000eb00330607008000eb0010002000dd
:106df0003006070011002000200020002d060700ab
:106e00008000eb00300020002a0607004000370019
:106e10008000eb000000eb002606070011002000b8
:106e20001000200023060700110020002000200091
:106e3000200607008000eb00300020001d06070040
:106e400033003700110020000000eb001906070096
:106e5000110020001000200016060700110020007d
:106e600020002000130607008000eb003000200007
:106e700010060700260037008000eb000000eb0042
:106e80000c0607008000eb00100020000906070038
:106e90008000eb0020002000060607001100200003
:106ea0003000200003060700190037001100200001
:106eb0000000eb00ff0507008000eb001000200041
:106ec000fc0507008000eb0020002000f90507000a
:106ed0001100200030002000f60507000c003700ec
:106ee000110020000000eb00f20507001100200057
:106ef00010002000ef0507001100200020002000f6
:106f0000ec0507001100200030002000e905070013
:106f10000080fa00000006001000fa0070079800d8
:106f20000000eb00600798000000eb00500798009d
:106f30000000eb00400798000000eb0030079800cd
:106f40000000eb00200798000000eb0010079800fd
:106f50000000eb00000f78000000eb004007070086
:106f600060079800100020003d07070050079800b8
:106f7000200020003a070700400798006e009000ac
:106f8000300798005e009000000040002007980045
:106f90004e0090004200dd0010079800be009000f7
:106fa0002e009000808040001e00900080804000f5
:106fb0007e0090000088b900000f78001e00780065
:106fc0000080fa00000006000400fa001007980094
:106fd00050002000000f78001e0078000080fa00aa
:106fe000000006002000fa00200f9800310f9800e2
:106ff0000000eb00100f98000000eb00000f98005d
:107000000000eb00700798000000eb00600798009c
:107010000000eb00500798000000eb0040079800cc
:107020000000eb00300798006000b80010079800df
:10703000210798000000eb00000f78002e08900058
:10704000e70f500039003c0080002000000f78005e
:107050002e089000600f98006e089000e30f50001b
:10706000230032006e089000e30f50000a003c003d
:107070006e089000e10f5000170032006e0890007b
:10708000e10f500017003c006e0890000000e00087
:107090000e0032008f0037006e089000e50f5000a0
:1070a000190032006e089000e50f50001300350003
:1070b0006e089000e60f5000160032006e08900037
:1070c000e70f5000160032008200370060082000f1
:1070d0003007980035003700600c2000300798001a
:1070e0003200370060092000300798002f00370079
:1070f000600d2000300798002c003700600a200047
:107100003007980029003700600e200030079800f3
:1071100026003700600b200030079800230037005e
:10712000600f2000300798002000370090002000fa
:10713000000f78002e089000700f98007e089000d5
:10714000e10f5000110032007e089000e10f500066
:1071500004003c007e0890000000e00008003200bf
:107160005c0037007e089000e20f50000a003200f9
:107170007e089000e30f50000a00320055003700ef
:10718000600920003007980008003700600a2000de
:107190003007980005003700600520003007980090
:1071a00002003700600d2000300798008000eb00df
:1071b0001e0078003f05070060c2a90020002000e3
:1071c000540d0700000000003e009000510d070024
:1071d0000000eb004f0d0700100f98000000eb00bf
:1071e0004c0d0700000f98000000eb00490d070050
:1071f00070079800110020001e0078002d05070080
:107200001e089000600798006e0090004800dd00a6
:10721000600798008e089000f00f200080806000ca
:107220006e00900001007000600798006e009000f2
:1072300000004000600798007e0090004700de00dc
:10724000700798000000eb00500798005e00900067
:107250004800dd0050079800fe009000f00f20006d
:10726000808060005e009000010070005007980070
:10727000ee0090005e0090000080700040079800d3
:107280004e0190008000eb002e089000ec000700fb
:107290003e099000ce0090002e089000490807009b
:1072a000cf80de00cff30700100798002107980079
:1072b0001e019000ae0190002e0890000a00070009
:1072c0001e009000ae009000400f9800510f9800f3
:1072d00001003700020037004e089000de089000e1
:1072e0000080fa00000006007000fa00889fbe00cf
:1072f0008a1f7800503798006237980073379800db
:1073000040062000400798006a00470041e32a0039
:1073100017000900311878000003b1006000b800c0
:107320002007980031079800a00320000e004000bd
:1073300042e02a0017000900321878000003b1006b
:107340000000eb00100798000000eb00000f780031
:107350005e309000800040000080200000804000ef
:10736000900078004e009000808f50003000350073
:107370000000eb00000f7800130037005e32900031
:107380009e027800de3090001e01e80040062000da
:107390000088b90002004000c200dd0080812000aa
:1073a000008040001001be004006200000a0b9008f
:1073b00005004000c200dd00808120000080400008
:1073c0000288be001e0fe8004e0090009e0f1000c5
:1073d000eaff3500de3090004e0090000001e90029
:1073e000818040000080200000804000020878007a
:1073f000de3190005e309000800040000080200070
:107400000080400010017800400620000098b9007c
:1074100002004000c200dd008081200000804000aa
:107420006e319000fe3190000288be000f003700e0
:10743000de3190005e30900080004000008020002f
:107440000080400010017800400620000098b9003c
:1074500002004000c200dd0080812000008040006a
:107460006e319000fe3190000288be000000eb00fb
:10747000100798001b0037005e3490005e309000cb
:10748000a10320008e8040004200dd00010040008a
:107490001002be00de3090001e0190004006200069
:1074a0000088b90002004000c200dd008081200099
:1074b000008040001001be000400be0075f307000c
:1074c0000001be00a10320008e8040004240dd008c
:1074d000010040000288be001e0090000000e8008d
:1074e000100798005e30900080004000008020006f
:1074f00000804000900078001e009000808f5000b7
:10750000ddff3d005e3590005e309000a10320005d
:107510008e8040004200dd00010040001004be00eb
:107520005e3090008000400000802000008040001d
:10753000100078000000e800cf80de0029f307008b
:107540000001be000800be00aff307000001be004e
:10755000ea0047004250dd00010040000288be0002
:10756000de309000018140000080200000004100da
:10757000100078000001e8008180400000802000b9
:1075800000804000020878005e309000ea0047006a
:107590004200dd00010040001001be0022079800fb
:1075a000330798002e019000be0190005e309000dd
:1075b000040007004f0578004f04be000080fa0069
:1075c000000006000a00fa00200798003207980021
:1075d000430798006000b800008fbe0002002c0036
:1075e000934724003e009000ce009000c8f30700af
:1075f0000000e00001003200070037002e0090007c
:10760000c200dd0080ad210000804000301f780006
:1076100020177800070037002e009000c200dd0020
:1076200080ad2100008040003e019000ce0190001e
:107630000288be001e00be000080fa0000000600a6
:107640000800fa00100798002107980032079800f8
:107650000000eb00000f78002e009000e10f5000ba
:1076600006003a001e0090008000400080b021001b
:1076700000804000100f7800060037001e009000c8
:107680008000400080b0210000804000be009000db
:10769000010878001e0078000080fa000000060053
:1076a0001000fa00500798000000eb004007980017
:1076b0000000eb00300798000000eb002007980066
:1076c0006000b800008fbe005e009000e70f500021
:1076d00002003400700020005007980060c2a9002a
:1076e0005e00900062fd07000000eb00090c07003f
:1076f000400798000000eb00060c070030079800d8
:1077000000000000a000200059fd07004e0090007e
:10771000200798002e0090004500dd00200798000b
:10772000be009000800f20000080600030079800ad
:107730003e0090004300de0030079800be0090003d
:10774000f00f2000808060002e009000010070008b
:10775000200798002e009000cf80de00a1f20700e5
:1077600060079800710798002e0090000000e0006c
:1077700007003d0002002000037824006e00900006
:10778000fe009000c3f207006007980071079800a0
:107790000200200003e823006e009000fe0090002d
:1077a0005df30700008fbe001e01be005e0090006a
:1077b000030007001e00be000080fa000000060063
:1077c0004e00fa00889fbe008a1f7800402798006c
:1077d00052279800632798006800470041e82a0074
:1077e0000f000900311878000002b1006000b800f5
:1077f0002007980031079800800220000e0040000a
:1078000042e62a000f000900321878000002b10099
:107810000000eb00100798000000eb00000f78005c
:107820004e2090008000400000b221000080400007
:1078300010007800f30f50002c0034000000eb0023
:10784000000f7800110037004e2290009e02780051
:107850004e2090001e01e8007400b90002004000b4
:10786000c200dd0000b32100008040001001be0016
:107870007420b90005004000c200dd0000b3210003
:10788000008040000288be001e0fe8003301200087
:107890009e8f1100ecff34004e20900080004000cd
:1078a00000b2210080804000300120008008780074
:1078b000ce2190004e2090008000400000b22100b8
:1078c00000804000100178007418b90002004000e8
:1078d000c200dd0000b32100008040005e21900066
:1078e000ee2190000288be000e003700ce219000ed
:1078f0004e2090008000400000b221000080400037
:10790000100178007418b90002004000c200dd00c8
:1079100000b32100008040005e219000ee21900025
:107920000288be000000eb00100798001a00370024
:107930004e2490004e209000810220008e80400056
:107940004200dd00010040001002be004e20900009
:107950001e0190007400b90002004000c200dd006a
:1079600000b32100008040001001be000400be00f2
:1079700048f207000001be00810220008e80400016
:107980004240dd00010040000288be001e00900061
:107990000000e800100798004e2090008000400092
:1079a00000b2210000804000900078001e0090008e
:1079b000808f5000deff3d004e2590004e2090004d
:1079c000810220008e8040004200dd000100400066
:1079d0001004be004e2090008000400000b2210044
:1079e00000804000100078000000e800cf80de003a
:1079f000fcf107000001be000800be0082f2070093
:107a00000001be00e80047004250dd0001004000d8
:107a10000288be00ce2090000181400000b221000b
:107a200000004100100078000001e8008180400063
:107a300000b2210000804000020878004e20900033
:107a4000e80047004200dd00010040001001be00d8
:107a500022079800330798002e019000be01900085
:107a60004e209000040007004f0578004f04be0030
:107a70000080fa00000006000a00fa0020079800c3
:107a800032079800430798006000b800008fbe00de
:107a900002002c00934724003e009000ce0090008e
:107aa0009bf207000000e0000100320007003700f1
:107ab0002e009000c200dd0000db210000804000ad
:107ac000301f780020177800070037002e00900044
:107ad000c200dd0000db2100008040003e0190007c
:107ae000ce0190000288be001e00be000080fa0099
:107af000000006000600fa00100798002107980011
:107b00000000eb00000f78001e0090000000e00075
:107b100003003a0010012000000f78000200370037
:107b200020012000000f78008000eb0040002000c2
:107b3000e00207001e007800f60a07002e00900001
:107b4000f40a07001100200040002000d9020700bd
:107b50000080fa00000006000400fa0010079800f8
:107b60008000eb0090002000d20207000000eb0034
:107b7000000f7800010037001e0fe80030062000db
:107b80009e0f1000fcff3400110020009000200028
:107b9000c80207000080fa00000006000200fa0098
:107ba000000f780040c2a9001e007800cc0a070030
:107bb0000080fa00000006000400fa0042c7bf007f
:107bc000804078000114a000014f78001e81fb0066
:107bd0006104200070052000237420008149780092
:107be00080497800824978004207a8001e00900072
:107bf00050052000303b8800a00a2000303b880060
:107c000027a6a80027e6a80027a6a9000080fa005a
:107c1000000006000e00fa00500798005e00900079
:107c2000504090008080fb001000200009020700f7
:107c3000300798005e009000604090008080fb005c
:107c40000000eb0003020700800078003e00900077
:107c500001004000300798005e0090003040900026
:107c60008080fb0010002000fa0107002007980028
:107c70005e009000404090008080fb000000eb0020
:107c8000f4010700800078002e0090000100400001
:107c9000200798005e009000104090008080fb005c
:107ca00010002000eb010700100798005e00900014
:107cb000204090008080fb000000eb00e501070001
:107cc000800078001e00900001004000100798001e
:107cd0005e009000104078008080fb000000eb0008
:107ce000dc010700000f78006e00900050052000b6
:107cf000303b8800a00a2000303b880027a6a8005f
:107d00007162200091407800c0cfb30000c06000d5
:107d100027e6b7003e009000203188007162200005
:107d200091407800c0cfb30000c060000004a00004
:107d300027e6b7002e0090002031880071622000f5
:107d400091407800c0cfb30000c060000014a000d4
:107d500027e6b7001e0090002031880027c6bf002c
:107d60003040b30027e6b7001e00780020318800bd
:107d700010002000400798007162200091407800b8
:107d8000c0cfb30000c0600027e6b70021318000fb
:107d90003e009000810f5000020032000000eb0016
:107da000400798007162200091407800c0cfb30076
:107db00000c060000004a00027e6b7002131800069
:107dc0002e009000810f5000020032000000eb00f6
:107dd000400798007162200091407800c0cfb30046
:107de00000c060000014a00027e6b7002131800029
:107df0001e009000810f5000020032000000eb00d6
:107e00004007980027c6bf003040b30027e6b70000
:107e1000203180009e0f1000020032000000eb00b5
:107e20004007980027a6a9004e0090000080fa00a5
:107e3000000006001000fa00600798007e00900025
:107e400050052000303b8800a00a2000303b88000d
:107e500027a6a8000000eb00500798005b00370041
:107e60007162200091407800c0cfb30000c0600074
:107e700027e6b700203180003007980071622000ab
:107e800091407800c0cfb30000c060000004a000a3
:107e900027e6b7002031800020079800716220009b
:107ea00091407800c0cfb30000c060000014a00073
:107eb00027e6b700203180001007980027c6bf00d2
:107ec0003040b30027e6b70020318000000f780073
:107ed000303180004b00de00610060000004e000f3
:107ee00004003200ee00900010c0b300f040980093
:107ef00003003700ee0090000040eb00f0409800d7
:107f00001000200040079800716220009140780026
:107f1000c0cfb30000c0600027e6b7002131800069
:107f20003e009000810f5000020032000000eb0084
:107f3000400798007162200091407800c0cfb300e4
:107f400000c060000004a00027e6b70021318000d7
:107f50002e009000810f5000020032000000eb0064
:107f6000400798007162200091407800c0cfb300b4
:107f700000c060000014a00027e6b7002131800097
:107f80001e009000810f5000020032000000eb0044
:107f90004007980027c6bf003040b30027e6b7006f
:107fa000203180009e0f1000020032000000eb0024
:107fb000400798004e0090000000e00006003a00e4
:107fc0005e0090000000e800500798005e009000fe
:107fd000e20f5000a2ff340027a6a9004e00900037
:107fe0000000e0002b0032009e0078000000eb0053
:107ff00039010700804078006e0090000148780049
:108000009e0090001000200033010700804078009f
:108010006e009000114098009e0090000000eb0060
:108020002d010700804078006e00900021409800ec
:10803000ae0090001000200027010700804078006b
:108040006e00900031409800ae0090000000eb0000
:1080500021010700804078006e00900041409800a8
:10806000be009000100020001b0107008040780037
:108070006e00900051409800be0090000000eb00a0
:1080800015010700804078006e0090006140980064
:1080900018003700ee0090000040eb0080487800a8
:1080a000ee0090000040eb0090409800ee00900041
:1080b0000040eb00a0409800ee0090000040eb0074
:1080c000b0409800ee0090000040eb00c0409800e7
:1080d000ee0090000040eb00d0409800ee009000d1
:1080e0000040eb00e0409800ee0090000040eb0004
:1080f000f04098004e0090000080fa00000006005a
:108100001200fa0040079800510798004e009000b6
:10811000304090000080fb00600798006e009000e7
:10812000e30f500029003200ee009000e38f500072
:108130000a003c006e019000e10f51001700320070
:10814000ee019000e18f51001a003c006e0090009b
:108150000000e0000b00320034003700ee00900019
:10816000e58f5000250032006e019000e50f5100b0
:108170001c003500ee019000e68f51002500320012
:108180002a0037005e00900041ea2a00080009003a
:10819000315878009000b100290037005e0090004f
:1081a000d2ea2a0008000900325878009000b10095
:1081b000230037005e00900063eb2a0009000900ed
:1081c00033587800a000b1001d0037005e00900019
:1081d00001ec2a000b00090031587800c000b10002
:1081e000170037005e009000c2ec2a000a00090068
:1081f00032587800b000b100110037005e009000e6
:1082000073ed2a0008000900335878009000b1008f
:108210000b0037005e00900001ee2a000a00090002
:1082200031587800b000b100050037005e009000c2
:10823000b2ee2a000a00090032587800b000b100fe
:108240004e009000104090000080fb006101b900da
:108250000080eb008080eb00020140008381480039
:1082600072079800030f9800b00020000100200062
:108270007e0190008e099000800f5100818f59007f
:108280003f003e007e0090008e08900000600100dc
:108290000b0037000e0037001100370014003700c4
:1082a000170037001a0037001d0037002000370084
:1082b0002300370026003700290037002c00370044
:1082c00061ef2a005e00900094e107002f00370064
:1082d000f1ef2a005e00900090e107002b003700cc
:1082e00091f02a005e0090008ce107002700370023
:1082f00001f12a005e00900088e1070023003700aa
:1083000071f12a005e00900084e107001f00370031
:10831000c1f12a005e00900080e107001b003700d9
:1083200021f22a005e0090007ce107001700370070
:1083300081f22a005e00900078e107001300370008
:1083400001f32a005e00900074e107000f0037007f
:10835000b1f32a005e00900070e107000b003700c7
:1083600041f42a005e0090006ce10700070037002e
:10837000e1f42a005e00900068e107000300370086
:1083800081f52a005e00900064e107004e00900035
:10839000204090000080fb00801f780040f62a00fb
:1083a000801f78000e00780021e10700e487570065
:1083b0008e0078005e00900058e107004e009000ab
:1083c000104078000080fb00801f7800b0f62a0083
:1083d000801f78000e00780015e10700e487570041
:1083e0008e0078005e0090004ce107001000200035
:1083f0000080fa00000006000400fa00000f780078
:10840000110798001e007800604090000081fb007a
:108410001e007800504090008080fb001e00780015
:10842000404090000080fb00821f7800811f780090
:10843000801f780020f72a00801f78001e0090001f
:10844000fbe00700e8875700100020000080fa00da
:10845000000006000800fa00200798003107980085
:108460003e009000a2002000110009000280d80008
:10847000104798003e009000004178001e40900098
:108480000080fb006a00b900004f51001e409000c0
:108490000080fb00100798001e0090004400dd00e3
:1084a000100798009e80fb001e0090000100400015
:1084b000100798002e0090000000e000030032003a
:1084c0001e0090004800dd00100798001e0090007c
:1084d0000080fa00000006000a00fa003007980049
:1084e000410798003e0090000000e00008003200c4
:1084f000ce00900000f02f00008060001007980070
:108500001e0090004800de001007980004003700ad
:108510004e009000f10f200001006000100798004d
:108520001e0090008040780000cfb30000c06000c3
:10853000104798001e4090000080fb004400de00c1
:10854000104798001e0090006f4f60001e40900082
:108550000080fb00200798002e0090006a00b90000
:10856000200798009e80fb002e0090000100400034
:10857000200798002e0090000080fa0000000600fe
:108580000000fa002c03a8002c23a8002c43a8000c
:108590002c63a8002c83a8002ca3a8002cc3a8003f
:1085a0002ce3a8002d03a8002d23a8002d43a8002c
:1085b0002d63a8002d83a800c8a2a900c8c2a900e5
:1085c000c8e2a900c9e2a900c902a900d002a90015
:1085d000d022a900d042a900d062a900d0a2a9004f
:1085e000d0c2a900d0e2a900d102a900d122a900dd
:1085f000c002a800c022a800c082a800c0e2a80053
:10860000c102a800c122a800c142a800c9a2a800b6
:1086100069a0a900c9c2a800c922a800d082a800e8
:1086200000000000d4c2a80000000000d4e2a800ae
:1086300000000000d502a80000000000d522a8001c
:1086400000000000d402a80000000000d462a800ce
:1086500000000000cde2a80000000000d4a2a800a5
:1086600000000000cce2a80000000000d422a80016
:1086700000000000cca2a90000000000ccc2a900ac
:1086800000000000d442a900000000000000eb0040
:1086900020fc8800000000000000eb0020fc8800a7
:1086a000000000000000eb0020fc88000080fa00c1
:1086b000000006000800fa00000f7800110798007b
:1086c0001e0090000000e0000200320010002000b8
:1086d00010079800000000001e0078006101b9003a
:1086e0002207980033079800f000200001002000c6
:1086f0002e019000be019000800f5100818f590023
:108700009f003e002e009000be009000006001001f
:108710000f0037001900370020003700290037000c
:10872000330037003c003700460037004d0037006b
:10873000570037005e0037006800370072003700ce
:108740007c00370086003700880037008a00370039
:108750001e00900061406000614060004601dd0045
:10876000412d200091407800f0cbb30000c06000a4
:1087700002407000d4e2b700810037001e00900074
:1087800061406000c700dd00d4c2bf000074a100da
:1087900001407000d4e2b700790037001e0090005d
:1087a0006140600061416000512d200091407800df
:1087b000e0cfb30000c0600002407000d5e2b70017
:1087c0006f0037001e009000614060006140600053
:1087d00000414000512d200091407800d0cfb300df
:1087e00000c0600002407000d5e2b70064003700ae
:1087f0001e0090006140600061416000412d20003a
:1088000091407800e0cfb30000c0600002407000eb
:10881000d4e2b7005a0037001e00900061406000ab
:10882000614060004301dd00412d2000914078004f
:1088300070cfb30000c0600002407000d4e2b70007
:108840004f0037001e00900061406000c700dd004f
:10885000cdc2bf000074a10001407000cde2b7009e
:10886000470037001e0090006140600061406000da
:108870004501dd00412d200091407800f0cdb3008e
:1088800000c0600002407000d4e2b7003c00370036
:108890001e00900061406000c700dd00ccc2bf0038
:1088a0000074a10001407000cce2b7003400370032
:1088b0001e00900061406000614060000041400087
:1088c000412d200091407800d0cfb30000c060005f
:1088d00002407000d4e2b700290037001e0090006b
:1088e00061406000614060004501dd00c12c200056
:1088f00091407800f0cdb30000c0600002407000ed
:10890000cce2b7001e0037001e00900061406000fe
:10891000614060004601dd00c12c200091407800dc
:10892000f0cbb30000c0600002407000cce2b700a2
:10893000130037001e00900061406000614060003d
:108940004201dd00412d200091407800b0cfb300fe
:1089500000c0600002407000d4e2b7000800370099
:108960009e00900021fc8800050037001e01900049
:1089700022fc8800020037009e01900023fc880042
:108980000080fa00000006000800fa00000f7800de
:10899000000000000000eb0020fc88001e007800b2
:1089a0006101b9002207980033079800f000200009
:1089b000010020002e019000be019000800f5100a8
:1089c000818f590070003e002e009000be00900084
:1089d000006001000f003700150037001a00370053
:1089e0001e00370024003700280037002e00370013
:1089f00033003700390037003e00370044003700ad
:108a00004a00370050003700560037005800370042
:108a10005a003700d4c2bf000080fb004600de00d1
:108a2000614060000080fb0010079800580037008c
:108a3000d4c2bf000080fb004700de000080fb00c6
:108a40001007980052003700d5c2bf006140600097
:108a50000080fb00100798004d003700d5c2bf0012
:108a60000080fb000000d100614060000080fb003e
:108a70001007980046003700d4c2bf006140600074
:108a80000080fb001007980041003700d4c2bf00ef
:108a90000080fb004300de00614060000080fb00be
:108aa000100798003a003700cdc2bf000080fb00dd
:108ab0004700de000080fb001007980034003700fc
:108ac000d4c2bf000080fb004500de0061406000b2
:108ad0000080fb00100798002d003700ccc2bf00bb
:108ae0000080fb004700de000080fb0010079800bc
:108af00027003700d4c2bf000080fb000000d10077
:108b0000614060000080fb001007980020003700e3
:108b1000ccc2bf000080fb004500de006140600069
:108b20000080fb001007980019003700ccc2bf007e
:108b30000080fb004600de00614060000080fb001a
:108b40001007980012003700d4c2bf000080fb005d
:108b50004200de00614060000080fb0010079800ca
:108b60000b00370021fc8000110798000800370037
:108b700022fc8000120798000500370023fc8000cb
:108b800013079800020037000000eb001007980060
:108b90001e0090000080fa00000006000600fa00a7
:108ba0002007980010002000000f78000000eb0064
:108bb000100798000b0037002e0090001e00600088
:108bc000800078001e009000bafe07001e007800aa
:108bd00000004000000f78001e0090000000e80038
:108be000100798001e009000ef0f5000f2ff3400b5
:108bf0000080fa00000006000600fa0010002000c5
:108c0000100798000000eb00000f78000000eb0058
:108c1000200798000c0037002e0090005aff070034
:108c20000000e000020032001e0090001e0f400015
:108c30001e00900000004000100798002e009000d9
:108c40000000e800200798002e009000ef0f500071
:108c5000f1ff34001e0078000080fa0000000600da
:108c60000800fa00000f7800000000000000eb0090
:108c700020fc88001e0078006101b90022079800de
:108c800033079800f0002000010020002e01900022
:108c9000be019000800f5100818f590066003e0098
:108ca0002e009000be009000006001000f00370011
:108cb00013003700190037001f0037002500370068
:108cc000290037002f003700350037003a00370001
:108cd0004000370046003700480037004a003700a0
:108ce0004c0037004e00370050003700c3c2bf00b1
:108cf000614060000080fb001007980050003700c2
:108d0000c3c2bf000080fb000000d10061406000d2
:108d10000080fb001007980049003700c3c2bf0065
:108d20000080fb004200de00614060000080fb002c
:108d30001007980042003700cbc2bf000080fb0044
:108d40004500de00614060000080fb0010079800d5
:108d50003b003700c2c2bf00614060000080fb00e2
:108d60001007980036003700c2c2bf000080fb0029
:108d70000000d100614060000080fb0010079800f7
:108d80002f003700c2c2bf000080fb004400de009d
:108d9000614060000080fb00100798002800370049
:108da000c2c2bf000080fb004700de000080fb0065
:108db0001007980022003700cbc2bf000080fb00e4
:108dc0004600de00614060000080fb001007980054
:108dd0001b003700d2c2bf000080fb004400de0051
:108de000614060000080fb0010079800140037000d
:108df00021fc8000110798001100370022fc800040
:108e0000120798000e00370023fc8000130798001b
:108e10000b00370020fc8000100798000800370086
:108e200021fc8000110798000500370022fc80001b
:108e300012079800020037008001eb00130798002a
:108e40001e0090000080fa00000006000600fa00f4
:108e500010002000100798000000eb00000f7800c1
:108e60000000eb00200798000c0037002e00900057
:108e70007bff07000000e000020032001e009000af
:108e80001e0f40001e0090000000400010079800d8
:108e90002e0090000000e800200798002e009000af
:108ea000ef0f5000f1ff34001e0078000080fa0040
:108eb000000006000200fa000000eb00000f78003e
:108ec000270037009e0178001e0078004700dd0073
:108ed00080007800c0e6210000804000000178009a
:108ee00041e621004318dd0001004000020878003f
:108ef0001e00780041e621004300dd000080e8000c
:108f0000810040000000eb00800878001e0078001f
:108f100041e621004300dd00640040008100400084
:108f20000000eb00800878001e00780041e6210078
:108f30004300dd006600400081004000f007200093
:108f4000800878001e00780080004000c0ee2100fc
:108f5000808040000000eb00800878001e0fe800d1
:108f60001e00e000d7ff3400b00020004011880050
:108f700021e2a80020a2a9002062a9000040200050
:108f8000101188008560a9008580a900910a200041
:108f900091407800f0c8b30000c0600001c6b30083
:108fa00001407000a9e0b700a10a200091407800bc
:108fb00080cfb30000c060000014a000aae0b7009a
:108fc0009560a8009580a9000080fa0000000600c6
:108fd0000800fa0010079800210798001e00900072
:108fe000e10f5000010032000e0037004f0607006d
:108ff0001e0090004300dd008000780040e6210064
:1090000068005000808040002e009000eb050700b3
:10901000000f78004f0607001e0078003007980008
:1090200005003700ae0090000040eb00804878005b
:109030000000eb00300798003e0090000080fa002e
:10904000000006000800fa00100798004147980049
:109050001e009000e10f50000100320007003700b1
:1090600023c2bf000080fb000000d100614060000f
:109070000080fb00000f7800020037001000200085
:10908000000f78001e00e0000a003a001e00900069
:10909000e10f500001003200060037004e40900002
:1090a0000080fb002011880010002000300798008d
:1090b000020037000000eb00300798003e009000ef
:1090c0000080fa00000006000600fa001007980071
:1090d000210798000000eb00000f78000b0037001c
:1090e0001e007800800078002e0090000080400074
:1090f00010407800804078001e009000d1ff0700eb
:109100000000e000010032001e0fe8001e007800a1
:10911000800078002e009000008040001040780011
:109120000004e000eeff3a000000eb000080fa00cf
:10913000000006000600fa00100798001e009000cc
:10914000e10f5000010032000d003700f705070065
:109150001e0090004300dd008000780040e6210002
:109160006800500000804000c0050700000f780034
:10917000f80507001e00780020079800020037005d
:109180000000eb00200798002e0090000080fa00fd
:10919000000006000400fa00100798001e0090006e
:1091a000e10f5000010032000700370023c2bf006a
:1091b0000080fb000000d100614060000080fb00e7
:1091c000000f78000200370010002000000f780028
:1091d0001e0078000080fa00000006000400fa007b
:1091e000000f78001e007800e10f500001003200ef
:1091f000070037001e00780080004000c0ee21000c
:10920000008040001000780010079800020037002e
:109210000000eb00100798001e0090000080fa008c
:10922000000006000200fa00000f78001e0078001f
:10923000e10f500001003200060037001e007800e8
:1092400080004000c0ee2100808040000000eb0064
:10925000800878000080fa00000006000400fa0090
:10926000100798001e009000e10f5000010032002e
:1092700013003700ad0507001e0090004300dd001d
:109280008000780040e62100680050000080400027
:109290006c0507001e009000e10f50000300320033
:1092a0000600370030118000000f780022c2bf0096
:1092b000614060000004e000faff3a00a5050700e5
:1092c0000080fa00000006000200fa00000f78009b
:1092d0001e007800e10f500001003200040037004a
:1092e0002342a900000000002342a8000000000063
:1092f0000080fa0000000600809fbe000000fa0017
:1093000000f3800011f3800061004000e08048001d
:1093100000f3880011f388008580a9000080fa001e
:109320004f00be0000400600809fbe000000fa0013
:109330001c00370040e62100100090008000e8008b
:1093400040e62100300090008080600040e621006f
:1093500020009000808f500003003a001000200091
:1093600060f788000f00370040e621009000780089
:1093700040e6210010009000808040003011800005
:109380008048780040e62100100090008000e8004e
:1093900040e62100300090008080600040e621001f
:1093a0001100980022c2bf00614060000004e0008c
:1093b000e0ff3a008560a9000080fa004f00be007f
:1093c000004006004800fa00201f9800311f980056
:1093d000421f980064004700010a2b001700090093
:1093e000311878000003b1004e1990003227980020
:1093f000be219000e18f5100430032003e209000da
:10940000e20f50007c003200be2090000100e0001e
:1094100001003200b4003700640147000000200062
:1094200001f823000089be0064014700000020000d
:1094300001f82300200198003101980064014700e1
:109440000000200001f8230040019800510198001d
:10945000640147000000200001f82300600198002b
:1094600071019800640147000000200001f823000a
:1094700000099800110998006401470000002000cd
:1094800001f8230020099800310998006401470081
:109490000000200001f823004009980051099800bd
:1094a000640147000000200001f8230060099800d3
:1094b00071099800640147000000200001f82300b2
:1094c000001198001111980064014700000020006d
:1094d00001f8230020119800311198006401470021
:1094e0000000200001f8230040119800511198005d
:1094f000640147000000200001f82300601198007b
:10950000711198007d003700640147008000200041
:10951000018223000089be00640147008000200012
:109520000182230020019800310198006401470066
:109530008000200001822300400198005101980022
:109540006401470080002000018223006001980030
:10955000710198006401470080002000018223000f
:10956000000998001109980064014700800020005c
:109570000182230020099800310998006401470006
:1095800080002000018223004009980051099800c2
:1095900064014700800020000182230060099800d8
:1095a00071099800640147008000200001822300b7
:1095b00000119800111198006401470080002000fc
:1095c00001822300201198003111980064014700a6
:1095d0008000200001822300401198005111980062
:1095e0006401470080002000018223006011980080
:1095f000711198004100370064014700a00020006d
:1096000081ac23000089be0064014700a000200057
:1096100081ac2300200198003101980064014700cb
:10962000a000200081ac2300400198005101980067
:1096300064014700a000200081ac23006001980075
:109640007101980064014700a000200081ac230054
:10965000000998001109980064014700a00020004b
:1096600081a4230020099800310998006401470073
:10967000a000200081ac2300400998005109980007
:1096800064014700800020000182230060099800e7
:1096900071099800640147007000200001782300e0
:1096a000001198001111980064014700700020001b
:1096b00001782300201198003111980064014700bf
:1096c000700020000178230040119800511198008b
:1096d000640147008000200001822300601198008f
:1096e00071119800050037000200200003f82b00dc
:1096f00012279800232798001f0037002e1890008b
:10970000e40047004200dd00010040001001be00ff
:10971000721f9800032798003e189000cf80de004b
:10972000b0ea0700501f9800611f98003e18900093
:109730000000e00007003d00020020000378240044
:109740005e189000ee189000d2ea0700501f9800b3
:10975000611f98005e199000ee1990007e1890002d
:109760008e2090006ceb0700008fbe001e00be0034
:1097700010279800212798001e209000ae2090000e
:109780000080fa00000006000800fa00881f780038
:1097900010079800210798000000eb00000f7800e8
:1097a0001e009000104078000004e00003003a0022
:1097b0000000eb0030079800460037001e007800dc
:1097c000800078002e00900000804000104078005b
:1097d0000000fb003cdc0700000478001e0078005d
:1097e000800078001e00900000804000104078004b
:1097f0000000fb0034dc0700800f5400150032002d
:109800002e0090000000e800200798002e00900035
:10981000104078000004e00003003a000000eb0074
:10982000300798002b0037002e0090009040780001
:10983000c0c7b30080cf5000f1ff3a002e00900067
:109840000000e800200798000000eb00000f7800ff
:109850001b0037001e0fe8001e0078008000780013
:109860002e00900000804000104078000004e000ce
:10987000080032001e007800800078002e00900062
:109880000080400090407800c0c7b30080cf5000f7
:109890000b003a001e007800800078001e00900047
:1098a0000080400010407800520007000000e000f7
:1098b00003003a001e0078003007980005003700ca
:1098c000700220009e0f1000bcff34001e007800c4
:1098d000300798003e0090004f0478000080fa00a6
:1098e000000006000600fa00100798002107980003
:1098f0000080eb00000f78000e0037001e00900083
:10990000104178001e007800800078002e00900042
:109910000080400010407800804f510005003a0060
:109920001e0090000000e800100798000080eb0087
:10993000000f78001e0fe8001e00780080007800fd
:109940002e00900000804000104078000004e000ed
:10995000eaff3a001e0090000080fa0000000600b6
:109960000400fa00000f7800010d2b001e007800a3
:10997000dcff0700000f78001e00780090407800a0
:10998000d0c2b30080cf5000050032001e00780026
:1099900090407800b0c2b30080cf500001003a0080
:1099a0001e0fe800310d2b001e007800cdff0700d0
:1099b000000f7800510d2b001e007800c9ff070032
:1099c000000f78001e007800104078000004e000ce
:1099d000030032000000eb0010079800020037007f
:1099e00010002000100798001e0090000080fa0070
:1099f000000006000400fa00004f78001e00fb0083
:109a0000b8db07000000e00003003a00f0c5b30037
:109a10009e4f100003003a0010002000100798002d
:109a2000020037000000eb00100798001e009000b5
:109a30000080fa00000006000c00fa0020079800e1
:109a400031079800420798000000eb00000f7800f3
:109a5000010d2b002e009000a2ff070020079800a8
:109a60001e0037001e0078004200dd0080007800f4
:109a70003e00900000804000900078002e00900092
:109a800041ff0700100798001e0090000000e00052
:109a9000110032001e009000800078002e0090001f
:109aa00000804000010d2b008eff0700200798006a
:109ab0001e0078004200dd00800078003e0090002b
:109ac00000804000900090002e00900001000100f6
:109ad000500798000c0037001e0fe8001e007800a9
:109ae0004200dd00800078003e00900000804000d1
:109af00010007800104078000004e000d9ff3a0020
:109b00004e009000500798005e0090000080fa0020
:049b1000000006004b
:020000040000fa
:109b14007e1f000006000000000000000008000096
:109b240060160000000000003e1f0000400000001e
:109b340000000000841f000002000000000000007c
:109b4400ee1e0000500000000200000000000000b3
:109b54000000000000000000000000000000000001
:109b640000000000000000000000000000000000f1
:109b740000000000000000000000000000000000e1
:109b840000000000000000000000000000000000d1
:109b940000000000000000000000000000000000c1
:109ba40000000000000000000000000000000000b1
:109bb4000000000000000000861f000002000000fa
:109bc40000000000881f00000200000000000000e8
:109bd400601e00008e000000000000008a1f0000cc
:109be4004a000000020000000000210015110e00d0
:109bf4000d0c0b000b0a0a000909090009090800e9
:109c040008080800080808000707070007070700f6
:109c14000707070007070700073031003233340015
:109c24003536370038396100626364006566670061
:109c340068696a006b6c6d006e6f700071727300fe
:109c440074757600777879007a00000006210000a8
:109c540004000000020000000000000000000000fa
:109c6400e0200000120000000200000001000200d9
:109c7400000400000800100000000000202b2d004c
:109c840023300000fe200000080000000200000055
:109c9400686a6c00747a4c0000000000f220000036
:109ca4000c00000002000000686a6c00747a4c002a
:109cb400006343006e5b0000be2000002200000031
:109cc40002000000303132003334350036373800ba
:109cd400396162006364650066003000313233002c
:109ce4003435360037383900414243004445460094
:109cf400000000001e2000004800000002000000d8
:109d040000000000000000002440000000000000eb
:109d140000005900400000000000000088c340001b
:109d2400000000000084d7009741000080e0370065
:109d340079c3410043176e0005b5b500b8934600da
:109d4400f5f93f00e9034f00384d32001d30f900aa
:109d5400487782005a3cbf00737fdd004f157500c1
:109d64006620000032000000020000004e414e0058
:109d7400006e61006e0049004e460000696e660088
:109d84000030310032333400353637003839610061
:109d9400626364006566000030313200333435009c
:109da400363738003941420043444500460000003c
:109db4009820000026000000020000000a000800ad
:109dc4000a101000106469006f7578005870000064
:109dd40030313200333435003637380039616200af
:109de4006364650066414200434445004600000048
:109df4000a21000002000000020000000000000030
:109e04000c210000020000000200000030000000ed
:109e1400d41f00004a0000000200000000004100be
:109e240029211c0019171600151413001212110011
:109e34001111100010100f000f0f0f000e0e0e0066
:109e44000e0e0e000e0d0d000d0d0d000d30310027
:109e540032333400353637003839610062636400c8
:109e64006566670068696a006b6c6d006e6f7000f0
:109e74007172730074757600777879007a00000047
:109e84000e2100000200000002000000000000009b
:049e940000000000ca
:020000040000fa
:109e98000000fa000000eb00800888000000eb00da
:109ea80030088800f07f24006008880084e0a9005a
:109eb80094e0a80011e1a8000080fa000000060064
:109ec8000000fa00b30007000080fa000000060056
:109ed8000200fa00000f78001e00780010007800d9
:109ee8000080fa00000006000200fa00000f780067
:109ef8001e007800640007001e00780002000700ba
:109f08000080fa00000006000200fa00000f780046
:109f18001e0178006000b8003001980041019800e7
:109f2800960007001e017800100198002101980092
:109f38000080fa00000006000600fa0020079800da
:109f48008e000700008fbe002e00900010007800e1
:109f58000000e000230032002e009000a0009000d6
:109f680010009000be0f5000ae8f58000f00360052
:109f78002e00900030019000c00190002e0090004b
:109f8800a0009000100090003e024000ae82480001
:109f98000400be0002004000838048002e019000ab
:109fa80030019800410198000e0037002e00900003
:109fb80030019000c00190002e009000a000900099
:109fc800100090003e021000ae8218000400be008f
:109fd80002004000838048002e0190003001980064
:109fe800410198002e0090001e01be00120098004a
:109ff800230098002e00900030039000c0039000ca
:10a0080086007800a0002000000ab8006030b9007f
:10a0180005017800000141006a38b90000014100db
:10a02800820278000400be000080fa0000000600ea
:10a038000200fa00000f78001e007800beff07003b
:10a048009e00780010002000800878001e0078002c
:10a0580030039000c003900086007800a000200024
:10a06800000ab8006030b90005017800000141001d
:10a078006a38b90000014100820278000400be007d
:10a088000080fa00000006000200fa00000f7800c5
:10a098001e007800a8ff07009e0078000000eb0073
:10a0a800800878001e00780030039000c0039000fc
:10a0b80086007800a0002000000ab8006030b900cf
:10a0c80005017800000141006a38b900000141002b
:10a0d800820278000400be000080fa00000006003a
:10a0e8000600fa0020079800240007000001be00bf
:10a0f8002e00900001002000001f41000197490038
:10a108001e000700be0f5000ae8f5800fcff39003c
:10a118000080fa00000006000600fa0020079800f8
:10a1280016000700008fbe002e009000e90f5000b7
:10a13800080036002e009000a2002000110009003f
:10a148000280d800010020001e0f40005e974800e2
:10a158000400370010002000010020001e0f4000fe
:10a168005e97480005000700be0f5000ae8f5800ec
:10a17800fcff39000080fa00000006000000fa0029
:10a188000400070000fc800011fc80000080fa0039
:10a19800000006000200fa00f2fb800000fc8000cc
:10a1a80011fc8000000f51001e0078006101b8000a
:10a1b80000fc800011fc8000020040008380480001
:10a1c80000fc880011fc88000080fa0000000600ee
:10a1d800801f78000000fa000000eb0030088800bb
:10a1e800f0fb80000000e800f0fb880084e0a90094
:10a1f8000080fa004f007800004006008a00fa004c
:10a208000000eb00000f7800416a200091407800c0
:10a2180000ceb30000c060009040b300a4e6b700d1
:10a22800816c20009140780000ceb30000c060002f
:10a238003040b300c8e6b700cff807001bfb0700a3
:10a24800ba00070012ff0700416a20009140780019
:10a2580000ceb30000c060009040b300a4e6b70091
:10a26800816c20009140780000ceb30000c06000ef
:10a278003040b300c8e6b700e600470000042b00f2
:10a28800801f780090042b00801f780050052b0059
:10a29800801f78000100780063d90700e68757001f
:10a2a800e60047001000200085fb0700600720003b
:10a2b8000e00400014ff0700600720000e00400059
:10a2c8005bff0700000820000e0040000eff07009b
:10a2d800000820000e00400055ff0700000037006e
:10a2e800600720000e00400013ff07000001be00b9
:10a2f800803e200001002000800f5100818f59000e
:10a3080003003600600720000e004000fefe070034
:10a31800000820000e00400007ff07000001be00f3
:10a328004006200001002000800f5100818f590055
:10a3380003003600000820000e004000f2fe07006f
:10a34800660047002e0007000000e00003003a0006
:10a3580030002000200798001000370066004700f2
:10a36800c1082b005dfd0700100798001e00900033
:10a37800104078000004e00003003a0020002000ac
:10a3880020079800050037004200200021fa2a0023
:10a398001e009000a6fd0700200798002e009000e0
:10a3a800e30f5000ceff32002e0090000000e000c6
:10a3b8000f0032002e009000e20f50000c00320017
:10a3c800600520000e004000ae009000811f78005c
:10a3d800f1082b00811f780013d90700e487570084
:10a3e800610520008e8040001000200034fb07002b
:10a3f800a1092b001000200031fb0700b8ff37002f
:10a408000800fa00300798000000eb0010079800d9
:10a41800e400470010002000ebfa07000000e0000d
:10a428003f003200ce4090001000200003fb0700e0
:10a438004e409000ed4f500003003a00a1c0b30019
:10a4480010002000fdfa07004e409000ed4f50002c
:10a458001a0032004e409000e84f50000d003200c4
:10a4680031fc8000f0042000808f500009003c007f
:10a4780032fc80004e40900080407800e0ee2100e1
:10a4880000004100014878000200e80030fc880024
:10a498000600370030fc80000000e00003003400b4
:10a4a80030fc80000000e90030fc8800be0090000d
:10a4b8000040eb00804878001900370010002000a9
:10a4c8001007980031fc8000e0ee210080804000f9
:10a4d8000040eb00804878000000eb00000f780097
:10a4e8000a0037001e007800800078003e009000c7
:10a4f800008140009e007800e0ee210000804000ce
:10a5080010407800004978001e0fe80030fc8000f9
:10a518009e0f1000f3ff34000000eb0030fc8800b1
:10a528001e0090000080fa00000006000000fa00fb
:10a538004382a9004362a9004342a9004322a9001b
:10a548004302a80042e2a90042c2a90042a2a9000f
:10a55800212420009140780030ceb30000c0600074
:10a5680042e2b70042c2bf003040b30042e2b70047
:10a5780045e2a90045c2a90045a2a9004422a900b4
:10a588004402a90041e2a8006382a9006362a9000d
:10a598006342a9006322a8006302a90062e2a9003d
:10a5a80062c2a90062a2a80021262000914078007a
:10a5b80030ceb30000c0600062e2b70062c2bf00e4
:10a5c8003040b30062e2b70065e2a90065c2a900a5
:10a5d80065a2a9006422a9006402a90061e2a8009a
:10a5e800811f7800821f7800831f78002174200063
:10a5f80062042000730520008248780083487800b0
:10a6080042c7a900cf0178004f017800cf00780039
:10a61800816a20009140780000ceb30000c060003d
:10a62800a040b300a8e6b700c16a200091407800b6
:10a6380000ceb30000c060000014a000ace6b70074
:10a64800916a20009140780000ceb30000c06000fd
:10a65800c040b300a9e6b700b16c20009140780073
:10a6680000ceb30000c060007040b300cbe6b70076
:10a67800316c20009140780000ceb30000c060002b
:10a68800a040b300c3e6b700416c200091407800b9
:10a6980000ceb30000c06000b040b300c4e6b7000d
:10a6a800811f7800821f7800831f780021742000a2
:10a6b80062042000730520008248780083487800ef
:10a6c80042c7a800cf0178004f017800cf0078007a
:10a6d8000080fa00000006000200fa00000f78006f
:10a6e8001e0078004012880040c2bf006140600030
:10a6f8000004e000fcff32000000eb00000f7800cf
:10a70800401280000080fa00000006000200fa00f3
:10a71800000f78001e0078004013880060c2bf0058
:10a72800614060000004e000fcff32000000eb0024
:10a73800000f7800401380000080fa000000060037
:10a748000600fa00004f7800110798001e009000dc
:10a75800440007000000e000030032000000eb00a6
:10a7680020079800100037001e0090009000780025
:10a778001e00900010009000008040001e487800e5
:10a788001e009000100090008000e8001e0090005d
:10a7980030009000808060001e009000110098003a
:10a7a80010002000200798002e0090000080fa007a
:10a7b800000006000600fa00000f78001107980054
:10a7c8001e0090003b0007000000e0000600320079
:10a7d8009e0078000040eb00804878000000eb0005
:10a7e80020079800120037001e00900090007800a3
:10a7f8001e009000200090000080400090407800eb
:10a808001e007800014878001e009000200090008b
:10a818008000e8001e0090003000900080806000fa
:10a828001e009000210098001000200020079800ca
:10a838002e0090000080fa00000006000200fa00d6
:10a84800000f78009e0078000000eb00a000980040
:10a858009e0078000000eb00900098000080fa004d
:10a86800000006000400fa00000f78001e007800bf
:10a87800100090008000e8001e0078003000900072
:10a88800808060001e00780020009000808f5000bb
:10a8980003003a001000200010079800020037005b
:10a8a8000000eb00100798001e0090000080fa00de
:10a8b800000006000400fa00000f78001e0078006f
:10a8c800a00090001e00780010009000808f5000bb
:10a8d80003003a001000200010079800020037001b
:10a8e8000000eb00100798001e0090000080fa009e
:10a8f800000006000200fa00000f78001e00780031
:10a90800900090001e007800200090008080500089
:10a918001e00780030009000008060000080fa007f
:10a92800000006000000fa0040fc80000000e00083
:10a9380001003a00ff3ffc0040fc80000000e800f6
:10a9480040fc88000080fa00000006000000fa00c1
:10a9580040fc80000000e90040fc880040fc8000ca
:10a968000000e00001003a000000fc000080fa004e
:04a9780000000600d5
:020000040000fa
:04a97c000000fe00d9
:00000001FF
